:0401CB00AA82AB83D6
:0E01CF008A828B83E493FCA3AA82AB83ECFDAF
:0E01DD00600F8D82C002C0031216AFD003D097
:0301EB000280E1AE
:0101EE0022EE
:0601EF0090732E0201CB0B
:0B01F50012179AE58260069073321228
:0202000001CB30
:040202007808E4F2A2
:0D02060012171A121748AA82BA08028003C4
:03021300BA7F1699
:0C0216007808E260EB12179AE5826003A2
:030222001201EFD7
:070225007808E214F280DA10
:03022C00BA1516EA
:0C022F007808E260D212179AE5826003A2
:03023B001201EFBE
:07023E007808E214F280EAE7
:05024500BA0D027A0A67
:0E024A00BA0A0F12179AE582603775820A12FF
:0402580016AF802F2E
:06025C007808E2B42E0058
:0A02620050A27808E2FB780804F2CD
:0A026C00EB24F4F582E434F0F5838E
:0E027600EAF0C00212179AE582D00260838A75
:07028400821216AF02020610
:0A028B007808E2FA780804F2EA2489
:0A029500F4F582E434F0F583740AF6
:0A029F00F07808E2FA780804F2EAA9
:0A02A90024F4F582E434F0F583E458
:0602B300F07809E4F222DC
:0802B9007806740AF278097955
:0B02C10008C3E3F5F0E295F050177859
:0902CC0009E2FA780904F2EA24BF
:0A02D500F4F582E434F0F583E0FA5A
:0302DF007806F2AC
:0102E20022F9
:0502E300AA82BA0A0026
:0A02E800500874302AF5820216AFA8
:0802F20074572AF5820216AFD1
:0E02FA00121748AA82C3EA648094B0401174BF
:0E030800B98AF063F08095F04006EA24D0F543
:02031600822241
:0E031800C3EA648094E1401174E68AF063F059
:0B0326008095F04006EA24A9F5822231
:0E033100C3EA648094C1401174C68AF063F080
:0B033F008095F04006EA24C9F58222F8
:09034A0078077401F275820022AB
:0E035300AA82AB838B82C002C003120369D062
:0803610003D0028A8202036945
:0E036900E582FAC4540FFB740F5BF582C002EC
:0D0377001202E3D002740F5AF5820202E375
:080384007806E2B42002800CAF
:08038C007806E2B409028004C6
:040394007A00800269
:020398007A01E8
:03039A008A822232
:0C039D00120384E58260051202B980F4AE
:0103A9002231
:0E03AA00AA82C3EA648094B0401174B98AF04C
:0D03B80063F08095F04006EA24D0F5822223
:0E03C500C3EA648094E1401174E68AF063F0AC
:0B03D3008095F0400674A92AF58222F4
:0E03DE00C3EA648094C1401174C68AF063F0D3
:0B03EC008095F0400674C92AF58222BB
:0403F7007582FF22EA
:0B03FB007800E4F208F212039D7A0083
:03040600BA020037
:0C04090050477806E2F582C0021203AAF8
:0C041500AB82D002EB30E70678077402DF
:02042100F222C5
:0C0423007800E2FC08E2C454F0CCC4CC29
:0E042F006CCC54F0CC6CFDEB3395E0FEEB4250
:0C043D0004EE42057800ECF208EDF2C07D
:09044900021202B9D0020A80B4CB
:010452002287
:0B0453007A017800E4F208F2C0021207
:04045E00039DD00228
:0C0462007806E2F582C0021203AAAB8209
:0C046E00D002EB20E7307800E2FC08E24E
:0E047A00C454F0CCC4CC6CCC54F0CC6CFDEB74
:0C0488003395E0FEEB4204EE42057800E4
:0E049400ECF208EDF27A00C0021202B9D002BA
:0204A20080BE1A
:0704A400EA60047807EAF2A8
:0104AB00222E
:0A04AC00C04CE581F54C2404F581F5
:0C04B6007A017802E4F208F208F208F281
:0704C200C00212039DD002ED
:0B04C9007806C3E2648094B050030288
:0204D400054DD4
:0C04D6007806C3E2F5F074B963F080957D
:0A04E200F040687802E2F56E08E2CF
:0904EC00F56F08E2F57008E2F575
:0B04F5007190000AE4F5F0126BA7A85C
:0C0500004C08A68208A68308A6F008F6A6
:0C050C007806E2FFE23395E0FBEF24D01C
:0C051800FFEB34FFFB3395E0FCFDA84C2A
:0E05240008EF26FFEB0836FBEC0836FCED086E
:0C05320036FD7802EFF208EBF208ECF264
:0D053E0008EDF27A00C0021202B9D00202EC
:02054B0004C9E1
:07054D00EA60047807EAF2FE
:0A05540078027900E2F308E209F3EF
:06055E00854C81D04C2207
:04056400AA82AB8339
:0C0568008A828B83E493FC60237806E217
:05057400B5040280093E
:0905790078077402F27582002279
:050582000ABA00010BA4
:0D058700C002C0031202B9D003D00280D41C
:040594007582012249
:090598001204537807E270467862
:0C05A1000FC2D575F007E230E704B2D5B8
:0205AD00F40454
:0E05AF00A430D50AF42401C5F0F43400C5F0E0
:0A05BD0024B7FA74F235F0FB74065F
:0C05C7002AF582E43BF5837800E2B400E2
:0A05D3000908E2B40004740180017D
:0105DD00E439
:0405DE00FAB401006A
:0405E200E433FAF014
:0105E60022F2
:0705E70012039D9073351211
:0705EE000564E582700122A3
:0D05F50012171A900064121F0975C90B90AF
:0B06020000C8121F097582080215F4E1
:0D060D00907A9FE493FA7B00C002C0039036
:0E061A00F36CE0C0E0A3E0C0E09000A4E49325
:0C062800C0E0740193C0E074CFC0E07427
:0A0634007FC0E07480C0E074BFC016
:0A063E00E0747FC0E07480C0E07437
:0A0648003BC0E07473C0E07480C092
:0C065200E0126CDAE58124F1F58174B748
:0B065E00C0E0747FC0E07480C0E07456
:0A066900A0C0E07473C0E07480C00C
:0B067300E0126CDAE58124FAF5812228
:04067E00780BE4F21F
:0A068200780B790AC3E3F5F0E29566
:04068C00F040012217
:0A069000780BE225E02424F582E453
:0A069A0034F1F583E0FBA3E0FC78E7
:0306A4000CE4F271
:0C06A700780CE275F004A4FEAFF02BF517
:0E06B30082EF3CF583E493FAA3E493FD4A70D2
:0406C1000302074EDB
:0E06C500EE2BFEEF3CFF8E828F83A3A3E49307
:0806D300F508A3E493F5098585
:0A06DB000882850983C003C00412E1
:0506E50001CBAE08AFDF
:0C06EA00097A808E828F838AF012728859
:0E06F600AA82D004D0038A057E000DBD00014B
:010704000EE6
:07070500ED2508F508EE35B3
:08070C0009F509742DC39AFAE6
:0E0714008A051AED6014758220C002C003C071
:0C072200041216AFD004D003D00280E611
:0A072E00850882850983C003C0041A
:0E0738001201CB75820A1216AFD004D00378DE
:080746000CE22401F20206A7F7
:09074E00780BE22401F20206829C
:080757007807E2B401028006FC
:06075F007807E2B4020D70
:0A0765009073B575F080126C677890
:03076F0007E4F2AA
:010772002264
:0A077300AA82AB83780AE2B40B00FF
:0E077D00400E758206C002C0031215F4D003B0
:02078B00D0029A
:0A078D00780AE2FC780A04F2EC2C72
:0A0797002424F582E434F1F583EA2E
:0507A100F0A3EBF022C3
:0707A6001201F51202B91265
:0907AD00039D7806E2FAC0021275
:0907B60002B9D002BA0D0280E77D
:0507BF00BA0A0280E20D
:0A07C40090F13AE4F0A3F0750A008A
:0A07CE00780AC3E2F5F0E50A95F0A1
:0507D800400302085A75
:0507DD00E50A250A24D5
:0A07E20024F582E434F1F583E0FC15
:0507EC00A3E0FD7E000A
:0A07F100EE75F004A4F50B85F00C82
:0C07FB002CF582E50C3DF583E493FFA390
:0B080700E493FB4F603DE50B2CFBE58C
:0C0812000C3DFF8B828F83A3A3E493FBBB
:0E081E00A3E493FF8B828F83E493FBB5021B50
:0A082C00E50B2CF582E50C3DF58389
:0E083600E493FBA3E493FF90F13AEBF0A3EF01
:03084400F080033E
:030847000E80A779
:0C084A0090F13AE0FBA3E0FC4B700505C8
:040856000A0207CEBD
:0E085A0090F13AE0FAA3E0FB4A6011C002C040
:0E086800038A828B8312008BD003D00280059E
:0508760078077402F296
:06087B001207570207A658
:070881009073C212077374AB
:08088800DAC0E07473C0E074F3
:08089000A6C0E07407C0E0906F
:0C089800F13C121C15E58124FCF58122C6
:04732E00082008002B
:037332003E2000FA
:0673350065626F6F740039
:0E733B006D616E7566616374757265722020F7
:0E73490020202025730A70726F647563742013
:0E73570020202020202020202025730A73658E
:0E7365007269616C2D6E756D6265722020205C
:0E7373002025750A63757272656E742D666C46
:0E7381006967687420202025750A6C6F672DDF
:0E738F00666F726D6174202020202020202562
:03739D00750A006E
:0E73A000736F6674776172652D76657273691E
:0773AE006F6E2025730A0039
:0D73B50053796E746178206572726F7200FA
:0273C2007E0645
:0273C400DE7376
:0273C600551F51
:0273C800E5736B
:0273CA00980524
:0273CC00ED735F
:0273CE00E705D1
:0273D000027445
:0273D2000D06A6
:0673D4001174000000002E
:0473DA00636D64007B
:0773DE003F0048656C7000E0
:0873E50054005461736B730046
:0E73ED0045203C30206F66662C2031206F6EEC
:0773FB003E004563686F00CE
:0E740200722065626F6F74005265626F6F7466
:01741000007B
:0A741100760056657273696F6E0015
:0C08A40012653578E4E2F58208E2F58385
:0E08B00008E2F5F008E2126936743BC0E0E49D
:0A08BE00C0E074B3C0E074F1C0E0C4
:0C08C80078E4E2F58208E2F58308E2F52E
:0E08D400F008E2121946E58124FCF5817582D8
:0708E20000122B67026927D9
:0708E90090F1EE121534122C
:0608F00008A490F1EE02E5
:0208F600159259
:0E08F80090F1C6E0FAA3E0FBA3E0FCA3E0FD54
:0E09060090F1E5E0FEA3E0FFA3E0F8A3E0F926
:0E091400C002C003C004C0058E828F8388F02D
:0E092200E9123D2AAA82AB83ACF0FDE58124E8
:0E093000FCF58190F1D0EAF0A3EBF0A3ECF01F
:04093E00A3EDF02213
:06094200780DE2600122C5
:0C094800126535743BC0E0E4C0E074B3FD
:0A095400C0E074F1C0E078E4E2F5C1
:0E095E008208E2F58308E2F5F008E212182D97
:0E096C00E58124FCF58190F1B3E0FABA0102B6
:02097A00803CBF
:0C097C0090F1B37401F090F1B4E4F0903D
:0C098800F1B574FAF0A3E4F0756E007590
:060994006F09E4F570900C
:06099A00F1BA1252177AB7
:0409A0001B7B748ABF
:0409A4006E8B6F7572
:0609A8007006E4F57190F9
:0609AE00F1BA1251E290C3
:0409B400F1B9E4F0C1
:0B09B80090F1B4E0FABA1503020AA5A2
:0309C300BA010076
:0709C600500590F1C3E4F0BD
:0309CD00BA02006B
:0E09D000500E90F1B7E4F0A3F090F1C4E4F003
:0209DE00A3F084
:0309E000BA030057
:0E09E30050209000A6E493FB740193FC740274
:0E09F10093FD740393FE90F1C6EBF0A3ECF0BF
:0609FF00A3EDF0A3EEF0F1
:030A0500BA040030
:0E0A0800500E90F1CAE4F0A3F0A37403F0A323
:020A1600E4F00A
:030A1800BA05001C
:070A1B00500590F1CEE4F05C
:030A2200BA060011
:070A2500500590F1CFE4F051
:030A2C00BA080005
:080A2F00500690F1D47401F0AF
:030A3700BA0900F9
:0A0A3A005013756E00756F10E4F59F
:070A44007090F1D5C0021211
:040A4B005217D0026C
:030A4F00BA0A00E0
:0E0A5200502E90F1B9E075F064A4FBE5F0FCC5
:0E0A60003395E0FDFE74762BFB74A13CFC7414
:0E0A6E00063DFDE43EFE90F1E5EBF0A3ECF05A
:060A7C00A3EDF0A3EEF073
:030A8200BA0B00AC
:090A8500500790F1E9E4F0A3F040
:030A8E00BA0D009E
:090A9100500790F1EBE4F0A3F032
:0B0A9A0090F1B47415F0780E7401F2B6
:090AA5001208F8780D7401F22228
:070AAE0090F1EE1215340275
:020AB5000942F4
:090AB700780E7401F290F1EE02D8
:020AC00015928D
:070AC200120AAE90F1EE02F2
:020AC900159284
:0A0ACB0074BAC0E074F1C0E0E4C0AA
:0A0AD500E07422C0E07474C0E07405
:0D0ADF0080C0E0126CDAE58124FAF5812276
:080AEC00756E00756F09E4F559
:050AF4007090F1EF120B
:070AF900521712039D7A0061
:080B00007806E2B40A02802627
:030B0800BA080028
:0C0B0B0050138A030AEB24EFF582E43457
:090B1700F1F5837806E2F0800597
:050B200078077401F2EA
:090B2500C0021202B9D00280D214
:060B2E007807E2600122DD
:050B3400120AAE756E0F
:030B3900EF756FE6
:060B3C00F1757009E4F5FB
:050B42007190F1BA12F0
:050B470051E2020AB7B3
:0E0B4C0090F1E5E0FAA3E0FBA3E0FCA3E0FDDE
:0C0B5A00C002C003C004C0057432C0E03B
:0C0B66007474C0E07480C0E0126CDAE52A
:060B72008124F9F5812247
:090B78001204AC7807E2600122CE
:070B8100120AAE90F1E578C5
:0C0B880002E2F0A308E2F0A308E2F0A3F0
:0A0B940008E2F01208F8120AB70296
:020B9E004DF513
:0D0BA00090F1B5E0FAA3E0FBC002C00374C1
:0A0BAD0042C0E07474C0E07480C020
:0B0BB700E0126CDAE58124FBF58122DE
:090BC2001204AC7807E260012284
:070BCB00120AAE90F1B578AB
:0A0BD20000E2F0A308E2F0020AB707
:0E0BDC0090F1C4E0FAA3E0FB90F1B7E0FCA3B7
:0C0BEA00E0FDC002C003C004C005745A46
:0B0BF600C0E07474C0E07480C0E01226
:090C01006CDAE58124F9F5812289
:0A0C0A00C04CE581F54C2405F5818E
:0D0C1400AA82AB83ACF0C002C003C0047420
:0A0C210075C0E07474C0E07480C078
:0E0C2B00E0126CDAE58124FAF58112171A1234
:090C3900174890749A75F08012BE
:060C42006C6712171A9006
:090C4800749D75F080126C6712B6
:0C0C5100171A7A007D04A84C08E4F6088D
:0B0C5D00F608F608F6E54C2405F8A6A2
:010C68001A71
:070C6900EA4D7003020CE6E6
:0C0C70007B1A7CFF8B828C83C002C005C5
:0B0C7C00121E39D005D0028A038D043F
:0B0C8700EB4C60DEE54C2405F8E6B500
:040C92001A0280D3EF
:0B0C9600E54C2405F8E675F00EA424E0
:0A0CA10009FD74F535F0FE8D828E1A
:0E0CAB0083A3A3E0FDA3E0FE3395E0FFFAA8CB
:0C0CB9004C08ED26F6EE0836F6EF083683
:0C0CC500F6EA0836F6E54C2405F8E604D3
:0C0CD100FAE54C2405F8741F5AF61BBB12
:030CDD00FF011CF8
:060CE0008B028C0580A1CF
:0C0CE600A84C0808860208E6C313CA13D5
:0E0CF200CAC313CA13CAFB08E6030354C04B5F
:0E0D0000FBE6A2E713A2E7133395E08A828B8D
:070D0E0083854C81D04C22CB
:090D15001204AC7807E26001222F
:0C0D1E007800E2F5F008E245F070249047
:0D0D2A0074AC75F080120C0AAA82AB8390A5
:0E0D370074AF75F080C002C003120C0AAC82CB
:080D4500AD83D003D00280272A
:0C0D4D007800E2FE08E2FF8E028F03C077
:0C0D590002C0031204ACD003D0027807E3
:040D6500E260012225
:0B0D69007800E2FE08E2FF8E048F0518
:0E0D7400C3EA9CEB64808DF063F08095F04044
:0C0D82001EC004C005C002C00374B4C051
:0C0D8E00E07474C0E07480C0E0126CDA05
:070D9A00E58124F9F5812237
:0E0DA100C002C003C004C005120AAED005D0C7
:0E0DAF0004D003D00290F1B7EAF0A3EBF0906D
:0A0DBD00F1C4ECF0A3EDF0020AB758
:0C0DC70090F1C3E0FA7B00C002C003748E
:0A0DD300D6C0E07474C0E07480C064
:0B0DDD00E0126CDAE58124FBF58122B6
:090DE8001204AC7807E26001225C
:070DF100120AAE7800E29047
:060DF800F1C3F0020AB78E
:0D0DFE0090F1E9E0FAA3E0FBC002C003742D
:0A0E0B00F0C0E07474C0E07480C011
:0B0E1500E0126CDAE58124FBF581227D
:090E20001204AC7807E260012223
:070E2900120AAE90F1E97816
:0A0E300000E2F0A308E2F0020AB7A6
:0E0E3A0090F1C6E0FAA3E0FBA3E0FCA3E0FD0C
:0C0E4800C002C003C004C005740CC0E070
:0C0E54007475C0E07480C0E0126CDAE538
:060E60008124F9F5812256
:090E66001204AC7807E2600122DD
:070E6F00120AAE90F1C678F3
:0C0E760002E2F0A308E2F0A308E2F0A3FF
:090E820008E2F01208F8020AB7B8
:0E0E8B0090F1CAE0A3E0FBA3E0FCA3E0FD8B26
:0E0E990002ECC313CA13CAC313CA13CAFBED7B
:0E0EA700030354C04BFBED0303543FC002C0D5
:0A0EB50003741CC0E07475C0E07403
:0D0EBF0080C0E0126CDAE58124FBF5812291
:0C0ECC0078E1E2FA08E2C313CA13CAC3BB
:0E0ED80013CA13CAFB08E2030354C04BFBE22B
:0C0EE6000303543F78E5E2FC08E2C3136C
:0E0EF200CC13CCC313CC13CCFD08E203035485
:0E0F0000C04DFDE20303543FC002C003C00415
:0E0F0E00C0051204ACD005D004D003D0027888
:050F1C0007E260012264
:0E0F2100C002C003C004C005122F77E582D0C5
:0C0F2F0005D004D003D00260167433C05B
:0C0F3B00E07475C0E07480C0E0126CDA55
:070F470015811581158122BF
:0E0F4E00C3E49A74049B502FEA24FFFEEB3498
:0C0F5C00FFFF7800E2520608E25207EEA8
:0C0F68004F601AC002C0037463C0E07444
:0C0F740075C0E07480C0E0126CDAE5810A
:050F800024FBF58122B5
:0C0F85007800C3E2F5F0EC95F008E2F50E
:0C0F9100F0ED95F0501AC004C005748EFD
:0B0F9D00C0E07475C0E07480C0E0127A
:090FA8006CDAE58124FBF58122DD
:0C0FB100120AAE7800E2FA08E2FBE4FC51
:0E0FBD00EB2BCC33CC25E0CC33FDEA2A25E02B
:0E0FCB00FBEA232354034CFC7A0090F1CAEA9F
:0D0FD900F0A3EBF0A3ECF0A3EDF0020AB7DB
:0C0FE60090F1CEE0FA7B00C002C0037462
:0A0FF200A4C0E07475C0E07480C074
:0B0FFC00E0126CDAE58124FBF5812295
:091007001204AC7807E26001223A
:07101000120AAE7800E29025
:06101700F1CEF0020AB761
:0C101D0090F1CFE0FA7B00C002C0037429
:0A102900B5C0E07475C0E07480C02B
:0B103300E0126CDAE58124FBF581225D
:09103E001204AC7807E260012203
:0C104700120AAE7800E25401F208E4F254
:0C10530090F1CFE0FA7B007800E2B502DB
:08105F000708E2B5030280322C
:0E10670090F1B7E0FAA3E0FB90F1C4E0FCA327
:0E107500E0FD74FFC39CFC747F9DFD90F1B7FD
:0E108300ECF0A3EDF074FFC39AFA747F9BFBB0
:0810910090F1C4EAF0A3EBF0BA
:081099007800E290F1CFF002B3
:0210A1000AB78C
:0C10A30090F1D4E0FA7B00C002C003749E
:0A10AF00CAC0E07475C0E07480C090
:0B10B900E0126CDAE58124FBF58122D7
:0910C4001204AC7807E26001227D
:0710CD00120AAE7800E29068
:0610D400F1D4F0020AB79E
:0A10DA0012039D7806E2FAC002122C
:0610E40002B9D0027B00FE
:0E10EA00EB75F006A4FCFD9075DC93CDA3938E
:0910F800FEBD0005BE00028032BD
:0C1101008D828E83E493FDB50225EC2462
:0A110D00DCFCE43475FD8C828D8358
:0E111700A3A3E493FCA3E493FDC004C0058CE5
:0B112500828D8312008BD005D00422C5
:031130000B80B77A
:0611330078077402F222AD
:021139007A003A
:0E113B00EA75F006A4FBFC9075DC93CCA39340
:08114900FDBC0004BD00012201
:0E11510074012CFEE43DFF78808C828D838833
:0E115F00F0C002C003C006C007127288AC8246
:0E116D00AD83D007D006D003EC2EFEED3FFF81
:0E117B007C80EB9075DC93CBA393FD7880C055
:0C11890006C007C004C003C005C000740D
:0A11950036C0E07476C0E07480C03C
:0E119F00E0126CDAE58124F7F581D0020A0235
:0211AD00113BF4
:0B11AF00120AC290F1B4E0FA7B00903D
:0E11BA00F1B3E0FC7D00C002C003C004C0051C
:0A11C8007440C0E07476C0E074804B
:0D11D200C0E0126CDAE58124F9F5817A00A5
:0E11DF00EA75F006A4FBFC9075DC93CCA3939C
:0811ED00FDBC0004BD0001225D
:0A11F500EB24DCFBE43475FC8B8274
:0E11FF008C83A3A3A3A3E493FBA3E493FC4B74
:0D120D006013C002C003C0048B828C8312EA
:08121A00008BD004D003D002C8
:031222000A80BA85
:0D1225007A0090F1EEC002121534D002786C
:081232000EE260091208A47825
:05123A000EE4F27A0150
:0E123F0090F1EEC002121592D002EA60099002
:08124D00765775F080026C6712
:0912550090765D75F080026C6773
:06125E0090766D0207739B
:07741B004E3043414C4C00D0
:0E74220043616C6C7369676E3A2022257322F9
:027430000A0050
:0E7432004672657175656E63793A20256C644B
:027440000A0040
:0E7442004D61696E206465706C6F793A20258B
:0A74500064206D65746572730A0014
:0E745A00416363656C2063616C202B31673ADF
:0D746800202564202D31673A2025640A009C
:0E7475004F7269656E7420616E74656E6E6193
:0E74830020257320616E642070726573732083
:0974910061206B65792E2E2E009E
:03749A000D0A00D8
:0E749D0043616C6962726174696E672E2E2EF7
:0174AB0000E0
:0374AC00757000F8
:0574AF00646F776E0020
:0E74B400496E76616C696420616363656C3AB1
:0E74C200207570202825642920646F776E20C5
:0674D000282564290A00D2
:0E74D60041706F6765652064656C61793A20CE
:0C74E4002564207365636F6E64730A00FA
:0E74F00041706F676565206C6F636B6F75741C
:0E74FE003A202564207365636F6E64730A0084
:0E750C00526164696F2063616C3A20256C64E3
:02751A000A0065
:0E751C004D617820666C69676874206C6F673B
:09752A003A202564206B420A009E
:0E75330053746F72616765206D75737420620A
:0E7541006520656D707479206265666F7265F5
:0E754F00206368616E67696E67206C6F67204D
:06755D0073697A650A0063
:0E756300466C69676874206C6F672073697AE4
:0E75710065206D757374206265206D756C74F5
:0E757F0069706C65206F66202564206B420ADF
:01758D0000FD
:0E758E00466C69676874206C6F67206D6178C9
:08759C00202564206B420A0067
:0E75A40049676E697465206D6F64653A202535
:0375B200640A0068
:0E75B500506164206F7269656E746174696F55
:0775C3006E3A2025640A0066
:0E75CA00526164696F20656E61626C653A20E3
:0475D80025640A001C
:0275DC007576C2
:0275DE00C20BDE
:0275E000A00BFE
:0275E2009076A1
:0275E400E80DB0
:0275E600C70DCF
:0275E800AB7680
:0275EA00200E71
:0275EC00FE0D92
:0275EE00D17654
:0275F000780B16
:0275F2004C0B40
:0275F400EA7635
:0275F600EC0A9D
:0275F800CB0ABC
:0275FA0009770F
:0275FC00C410B9
:0275FE00A310D8
:027600003A77D7
:02760200660E12
:027604003A0E3C
:027606006577A6
:02760800150D5E
:02760A00DC0B97
:02760C008A777B
:02760E003E102C
:027610001D104B
:02761200BB7744
:02761400CC0E9A
:027616008B0ED9
:02761800D97720
:02761A00071057
:02761C00E60F77
:02761E000378EF
:04762000AF110000A6
:027624000A78E2
:047626002512000029
:02762A001C78CA
:0A762C00391100000000000000000A
:0A763600252D3230732025730A0061
:0E764000436F6E6669672076657273696F6EC0
:09764E003A2025642E25640A008F
:067657005361766564003A
:0E765D004E6F7468696E6720746F20736176DB
:02766B006500B8
:02766D00DA1031
:06766F002378000000007A
:0E7675006D203C6D65746572733E004D616959
:0D7683006E206465706C6F7920286D290001
:0E76900064203C64656C61793E0041706F6758
:0D769E0065652064656C6179202873290002
:0E76AB004C203C7365636F6E64733E0041704B
:0E76B9006F67656520646574656374206C6F8F
:0A76C700636B6F75742028732900AF
:0E76D10046203C667265713E0046726571751A
:0B76DF00656E637920286B487A290053
:0E76EA0063203C63616C6C3E0043616C6C730A
:0E76F80069676E2028382063686172206D611A
:03770600782900DF
:0E77090065203C302064697361626C652C2041
:0E7717003120656E61626C653E00456E6162F8
:0E7725006C652074656C656D65747279206109
:077733006E64205244460081
:0E773A0066203C63616C3E00526164696F2002
:0E77480063616C6962202863616C203D2072D1
:0E775600662F287874616C2F325E3136292937
:017764000024
:0E77650061203C2B673E203C2D673E004163B7
:0E77730063656C2063616C69622028302066BB
:097781006F72206175746F29001C
:0E778A006F203C3020616E74656E6E6120755C
:0E779800702C203120616E74656E6E6120646D
:0E77A6006F776E3E00506164206F7269656EF1
:0777B400746174696F6E003F
:0E77BB006C203C73697A653E00466C69676815
:0E77C90074206C6F672073697A6520286B420C
:0277D700290087
:0E77D90069203C30206475616C2C20312061E9
:0E77E700706F6765652C2032206D61696E3E03
:0E77F5000049676E69746572206D6F646500EF
:07780300730053686F77006A
:0E780A007700577269746520746F2065657091
:04781800726F6D001E
:07781C003F0048656C70009D
:0E78230063203C7661723E203C76616C756598
:0E7831003E0053657420636F6E666967202801
:0E783F003F20666F722068656C702C207320ED
:09784D00746F2073686F77290045
:0A126400C04CE581F54C2407F5812C
:0C126E00AA82E583FB30E7047A007B00D5
:0A127A00A84C08A603A84C0808A61B
:0C12840002087600A84C08E675F002A4F1
:0A1290002456F582747835F0F583DA
:0D129A00E493FDA3E493FE3395E0FFFCA870
:0C12A7004C0808E4C396FA74010896FB9A
:0912B3008A6EEBF56F3395E0F54E
:0A12BC0070F5718D828E838FF0ECC7
:0C12C600126BA7A84C08080808A68208B4
:0C12D200A68308A6F008F6A84C08E60465
:0A12DE0075F002A42456F58274781E
:0E12E80035F0F583E493FEA3E493FF3395E025
:0A12F600FAFBA84C0808866E088673
:081300006FE63395E0F570F58E
:0C130800718E828F838AF0EB126BA7AA13
:0C13140082AB83ACF0FDE54C2404F8EA49
:0E13200026FAEB0836FBEC0836FCED0836FD2D
:0E132E0074802AE43BFBE43CFCE43D8B828CA3
:07133C0083854C81D04C2297
:0E785600DB3DE43B143A6338CE365135EA335D
:0E786400963253312030FB2EE32DD72CD62B3D
:0E787200DF2AF029082926284B277626A6258E
:0E788000DB24152454239722DE212A217920AF
:0E788E00CC1F221F7B1ED81D381D9A1C001C0B
:0E789C00681BD31A401AAF19211996180C1840
:0E78AA008417FF167B16F9157915FB147F1451
:0E78B80004148B1313139D122812B5114311E3
:0E78C600D3106410F60F890F1E0FB40E4B0E78
:0E78D400E30D7D0D170DB20C4F0CEC0B8B0B62
:0E78E2002A0BCB0A6C0A0E0AB2095609FA08E4
:0E78F000A0084708EE0796073F07E906930633
:0E78FE003E06EA0596054305F104A0044F047A
:0E790C00FF03AF0360031203C40277022A02D6
:0E791A00DE0193014801FE00B4006A00220065
:0E792800D9FF91FF4AFF03FFBDFE77FE32FE3E
:0E793600EDFDA8FD64FD20FDDDFC9AFC58FC73
:0E79440016FCD4FB93FB52FB12FBD2FA93FA13
:0679520053FA14FAD6F905
:021343007A002E
:0E13450090FAA2E0FBFC700C90FAA2C002121B
:061353001E39D00280ECFF
:0E13590090FAA3C002C004121534D004D002D2
:08136700EC30E01A756EA4756C
:03136F006FFA759D
:061372007020E4F571900B
:0D137800F200C002C0041251E2D004D00205
:08138500EC30E11A756EC4752D
:03138D006FFA757F
:061390007020E4F57190ED
:0D139600F220C002C0041251E2D004D002C7
:0D13A30090FAA2E4F090FAA3C002C0041278
:0D13B0001592D004D002EC20E0030214B22C
:0B13BD0090F205E0FB20E4030214B2F4
:0C13C80090F1FA7892E2F0A308E2F090B5
:0A13D400F1F87447F090F213E09076
:0813DE00F1FCF090F214E09024
:0813E600F1FDF090F215E0901A
:0913EE00F1FEF090F1FFEBF0902C
:0A13F700F1F8C002C0041231449066
:0E140100F1F8744EF090F208E0FBA3E0FDA3BA
:0E140F00E0FEA3E0FF90F1FCEBF0A3EDF0A3F4
:0C141D00EEF0A3EFF090F1F812314490D3
:0E142900F1F87457F090F20CE0FBA3E0FDA385
:0E143700E0FEA3E0FF90F1FCEBF0A3EDF0A3CC
:0C144500EEF0A3EFF090F1F812314490AB
:0E145100F1F87448F090F206E0FBA3E0FD9085
:0E145F00F1FCEBF0A3EDF090F1FE74FFF0A3B2
:0E146D00F090F1F8123144D004D002EA70374A
:0E147B0090F205E0FB30E62F90F1F87459F086
:0914890090F210E090F1FCF090EB
:08149200F211E090F1FDF09071
:08149A00F212E090F1FEF09067
:0A14A200F1FFE4F090F1F8C004122D
:0614AC003144AA82D004C5
:0714B200EC20E103021345E9
:0B14B90090F225E0FBFC7003021345DD
:0814C40090F1F87456F07B0072
:0814CC00C3EB9C400302134531
:0A14D400EB2BFD2426F582E434F230
:0E14DE00F583E0FE7F0090F1FCEEF0A3EFF04E
:0A14EC00EE4F6024ED2426FDE434E9
:0C14F600F2FE8D828E83A3E090F1FFF0E7
:0E15020090F1F8C002C003C004123144D004BE
:04151000D003D00232
:031514000B80B594
:091517007458C0E07479C0E0745E
:0815200043C0E07413C0E09029
:0C152800F240121C15E58124FCF5812224
:0B7958006770735F7265706F727400DF
:0A153400AA82AB83E0FC850E8285DD
:0C153E000F83A3A3A3A3A3E0FDECB5055D
:0E154A000E758203C002C0031215F4D003D048
:011558000290
:07155900D21010AF02C21016
:0E1560008A828B83E060158A828B83C002C072
:07156E0003C022121E39D058
:0715750022D003D00280E444
:0A157C00850E82850F83A3A3A3A3AD
:0C158600A3E08A828B83F0A21092AF22B7
:0A159200AA82AB83E0FC850E82857F
:0C159C000F83A3A3A3A3A3E0FDECB505FF
:0315A80002800EB0
:0E15AB00758203C002C0031215F4D003D002F3
:0715B900D21010AF02C210B6
:0C15C0008A828B83E4F08A828B83C02235
:0615CC00121E77D022A2DE
:0415D2001092AF22A2
:0615D600AA827B007C00EC
:0815DC008A051AED60118C056F
:0715E4001DEDFC60F38B0418
:0815EB001CECFB60F40080F829
:0115F30022D5
:0415F400AA82C2AF56
:0C15F800758214C0021215D6D0027B05CB
:0E160400758201C002C00312491175824B129B
:0C161200400B7582011215D67582011282
:0C161E00491A75829612400B7582011269
:0E162A0015D6D003D002DBD2758200C00212AA
:0E163800400B7582021215D6D002EA30E62869
:0E164600758201C00212491175824B12400BD1
:0E1654007582281215D675820112491A758208
:0C1662000012400B75820A1215D6D0024F
:06166E00743F5AFB7C00F2
:08167400C3EC9B40030215F8D2
:0E167C00758201C002C003C0041249117582BC
:0E168A005E12400B75820A1215D6758201128F
:0C169800491A75820012400B75820A127C
:0B16A40015D6D004D003D0020C80C586
:0C16AF00AA82BA0A35780FE275F007A491
:0A16BB0024B7FBE434F2FC8B828CB0
:0E16C50083A3A3E0FBA3E0FCC002C003C004AB
:0A16D30074E3C0E07416C0E0C00329
:0616DD00C00475820D221D
:0616E300D004D003D00288
:0A16E900780FE275F007A424B7FBA8
:0C16F300E434F2FC8B828C83A3A3E0FBA8
:0C16FF00A3E0FCC003C0047415C0E0743C
:0A170B0017C0E0C003C0048A822268
:05171500D004D0032206
:0A171A00780FE275F007A424B7FA77
:0C172400E434F2FB8A828B83A3A3A3A30E
:0E173000E0FAA3E0FB4A600FC002C0038A8209
:09173E008B8312008BD003D00252
:01174700227F
:06174800C2AF780FE2FAC7
:0B174E00EA75F007A424B7F582E4342C
:0C175900F2F583E0FBA3E0FCC0028B82F1
:0E1765008C8312008BAB82AC83D002BBFF1EC4
:0C177300BCFF1B0A7810E2B502027A00ED
:0C177F00780FE2B502C990F2C5C002125A
:06178B001E39D00280BDF2
:09179100780FEAF2D2AF8B82223C
:0A179A00780FE275F007A424B7FAF7
:0C17A400E434F2FB74062AF582E43BF505
:0517B00083E0F5822238
:0A17B500C04C85814CAA82AB8378FA
:0C17BF0010E2B4020E758207C002C003E5
:0717CB001215F4D003D00257
:0A17D2007810E275F007A4FC24B7BC
:0C17DC00F582E434F2F583EAF0A3EBF0B0
:0A17E800EC24B7FCE434F2FA8C8222
:0C17F2008A83A3A3E54C24FCF8E6F0A3D6
:0C17FE0008E6F08C828A83A3A3A3A3E575
:0C180A004C24FAF8E6F0A308E6F074069F
:0C1816002CF582E43AF5837401F07810A0
:0A182200E2FA781004F28A82D04C3A
:01182C002299
:0A182D00C04C85814CC082C083C00E
:0A183700F0C0E0126535A84C0879F6
:0C184100DCC3E3F5F0E695F009E3F5F0F8
:0E184D0008E695F009E3F5F008E695F009E3EA
:0C185B00F5F008E695F05030E54C24FA5A
:0C186700F886060886077A007B00A84C73
:0E18730008EE26FEEF0836FFEA0836FAEB080C
:0C18810036FB78DCC3E29E08E29F08E220
:06188D009A08E29B5006E0
:06189300758200021940FD
:0B189900E54C24FAF8E6084670030254
:0218A400193DEC
:0A18A600A84C08860208860378E8C3
:0E18B000E224FFFC08E234FFFDEC5202ED5290
:0C18BE000378E8E2C39AFA08E29BFBE51D
:0C18CA004C24FAF8C3E69A08E69B500A8A
:0A18D600E54C24FAF88602088603A8
:0C18E000C002C003C002C003E54C24FCA1
:0C18EC00F8E6C0E008E6C0E0A84C088662
:0E18F800820886830886F008E6126891AC82AA
:0E190600E58124FCF581D003D002EC7004F5DD
:03191400828029A5
:0C191700E54C24FAF8E6C39AF608E69BBB
:0C192300F67C007D00A84C08EA26F6EBDC
:0E192F000836F6EC0836F6ED0836F602189982
:03193D00758201AF
:06194000854C81D04C2211
:0A194600C04C85814CC082C083C0F4
:0A195000F0C0E0126535A84C0879DC
:0C195A00DCC3E3F5F0E695F009E3F5F0DE
:0E19660008E695F009E3F5F008E695F009E3D0
:0C197400F5F008E695F05030E54C24FA40
:0C198000F886060886077A007B00A84C59
:0E198C0008EE26FEEF0836FFEA0836FAEB08F2
:0C199A0036FB78DCC3E29E08E29F08E206
:0619A6009A08E29B5006C6
:0619AC00758200021A59C9
:0B19B200E54C24FAF8E608467003023A
:0219BD001A56B8
:0A19BF00A84C08860208860378E8A9
:0E19C900E224FFFC08E234FFFDEC5202ED5276
:0C19D7000378E8E2C39AFA08E29BFBE503
:0C19E3004C24FAF8C3E69A08E69B500A70
:0A19EF00E54C24FAF886020886038E
:0C19F900C002C003C002C003E54C24FC87
:0C1A0500F8E6C0E008E6C0E0A84C088647
:0E1A1100820886830886F008E61267CBAC8256
:0E1A1F00E58124FCF581D003D002EC7004F5C3
:031A2D008280298B
:0C1A3000E54C24FAF8E6C39AF608E69BA1
:0C1A3C00F67C007D00A84C08EA26F6EBC2
:0E1A48000836F6EC0836F6ED0836F60219B24E
:031A560075820195
:061A5900854C81D04C22F7
:0A1A5F00C04CE581F54C2405F5812B
:091A69001204537807E260030245
:021A72001B2433
:051A7400A84C087600FB
:0A1A79007800E2FB08E2FC7D00A803
:0C1A83004C0808080808A60518A604185E
:0C1A8F00A603187600A84C0886077A0011
:0C1A9B007B007C00A84C0808EF26FFEA46
:0E1AA7000836FAEB0836FBEC0836FC7408C073
:0A1AB500E0E4C0E074C6C0E074F283
:0E1ABF00C0E08F828A838BF0EC12182DAA8271
:0C1ACD00E58124FCF581EA603CA84C088F
:0D1AD90086027B008A828B831203537A0001
:031AE600BA08003B
:0E1AE9005021758220C0021216AFD002EA24EE
:0A1AF700C6F582E434F2F583E0F551
:0B1B010082C002120369D0020A80DAE1
:061B0C0075820A1216AFFB
:081B1200A84C08B6F802800A95
:0A1B1A00A84C08740826F6021A7998
:061B2400854C81D04C222B
:091B2A001204537807E260012265
:0C1B33007800E2FA08E2FB7C008C058BD5
:0D1B3F00048A037A008A828B838CF0ED0209
:021B4C006936F8
:071B4E0012039D9079631260
:071B55000564E58270012226
:081B5C007A007B007C007D0093
:0C1B640078E4C3E2F5F0EA95F008E2F541
:0E1B7000F0EB95F008E2F5F0EC95F008E2F5E8
:0E1B7E00F0ED95F0502D8A828B838CF0EDC037
:0E1B8C0002C003C004C005126936D005D004A3
:0C1B9A00D003D00278E0E22AFA08E23B17
:0B1BA600FB08E23CFC08E23DFD80B3C0
:011BB1002211
:0C1BB20012653578DCE2FA08E2FB08E27C
:0D1BBE00FC08E2FDC002C003C004C00574B5
:0A1BCB0068C0E07479C0E07480C0C7
:0C1BD500E0126CDAE58124F9F58178E07B
:0E1BE100E2FA08E2FB08E2FC08E2FDC002C0E6
:0A1BEF0003C004C005747BC0E0745D
:0C1BF90079C0E07480C0E0126CDAE58175
:071C050024F9F58102699743
:071C0C00126A47907994026F
:021C1300077355
:05796300446F497400AF
:0E79680053746F726167652073697A653A2007
:05797600256C640A000D
:0E797B0053746F7261676520657261736520D9
:0B798900756E69743A20256C640A00DA
:02799400B21B24
:02799600A879CE
:027998005F1A74
:02799A00B779BB
:02799C002A1BA4
:02799E00CC79A2
:0279A0004E1B7C
:0679A200E4790000000082
:0E79A800660053686F772073746F72616765B5
:0179B60000D0
:0E79B70065203C626C6F636B3E0044756D7022
:0779C50020666C617368008D
:0E79CC007A203C626C6F636B3E004572617303
:0A79DA0065203C626C6F636B3E0099
:0E79E4005A203C6B65793E0045726173652048
:0E79F200616C6C2E203C6B65793E2069732021
:0E7A0000646F69742077697468204426490019
:0A1C1500C04C85814CAA82AB837499
:0C1C1F0010B50D0E758201C002C003124A
:061C2B0015F4D003D00205
:021C31007C0134
:051C3300EC60347D00AF
:0A1C3800C3ED950D5023ED2D24CED1
:0C1C4200F582E434F2F583E0FEA3E0FF3D
:0E1C4E008E828F83A3A3A3A3A3E0FEB504029E
:021C5C00800303
:031C5E000D80D71F
:061C6100EDB50D02800349
:031C67000C80C925
:0E1C6A008A828B83A3A3A3A3A3ECF074062AA3
:0C1C7800F582E43BF583E54C24FAF8E625
:0E1C8400F0A308E6F08A828B83E4F0A3F074EC
:0C1C9200082AFCE43BFDE54C24FCF8862D
:0E1C9E0006088607C002C0038E028C828D836A
:0E1CAC00EAF0A3AC82AD838F068C828D83EEAE
:0E1CBA00F0A3E4F0A37480F0A3AC82AD83D05D
:051CC80003D0027E0DB7
:0E1CCD008C828D83E4F0A3AC82AD83DEF38ABB
:0C1CDB00828B83A3A3A3A37411F0D2108A
:051CE70010AF02C21065
:051CEC00E50D250D24AB
:0A1CF100CEF582E434F2F583EAF048
:0A1CFB00A3EBF0050DA21092AFD08C
:021D05004C226E
:0E1D0700C0E0C0A8C082C083C0F0C002C0030C
:0E1D1500C004C005C006C007C000C001C0D099
:0A1D230075D000C04C74FFB5100726
:071D2D00E50D14F510802CF8
:0A1D3400E5812471FA850E82850F07
:0C1D3E0083A3A3A3A3EAF07408250EFB06
:061D4A00E4350FFC789067
:0E1D50008605088B828C83EDF0A3AB82AC83FA
:021D5E00DAF0B9
:0B1D600075818FE5116004D2AF800296
:021D6B00C2AF05
:021D6D00AA10BA
:051D6F000510E50DB5B3
:051D74001003751000D2
:051D7900E51025102417
:0A1D7E00CEF582E434F2F583E0F5BF
:061D88000EA3E0F50F853B
:0A1D8E000E82850F83E0FBA3E0FC4A
:081D9800BB0005BC0002804401
:0A1DA000850E82850F83A3A3E0FBEC
:0E1DAA00A3E0FC4B6022C0021253B1AB82AC2E
:0A1DB80083D002850E82850F83A3FD
:0E1DC200A3E0FDA3E0FEEBC39DFBEC9EFC3016
:021DD000E71218
:0A1DD200EAB51099E5117095D2AF43
:081DDC00758701C2AF021D6F03
:0A1DE400850E82850F83A3A3A3A33D
:0C1DEE00E0FA748F2AF5817408250EFBC2
:061DFA00E4350FFC7890B7
:0E1E00008B828C83E0FDA3AB82AC83A6050829
:0C1E0E00DAF0D04CD0D0D001D000D007CA
:0E1E1A00D006D005D004D003D002D0F0D08383
:0C1E2800D082D0E020E705C2AF021E36D9
:021E3400D2AF2B
:031E3600D0E022D7
:0A1E3900AA82AB83850E82850F8319
:0C1E4300EAF0A3EBF0121D07850E82856B
:0B1E4F000F83E0FAA3E0FB4A601A8555
:0A1E5A000E82850F83E4F0A3F085EB
:0A1E64000E82850F83A3A3E4F0A310
:051E6E00F07582012265
:041E73007582002252
:061E7700AA82AB837C008F
:0A1E7D00C3EC950D502CEC2C24CE84
:0C1E8700F582E434F2F583E0FDA3E0FEF8
:0E1E93008D828E83E0FFA3E0F8EFB5020CE82D
:0B1EA100B503088D828E83E4F0A3F0EF
:031EAC000C80CED9
:011EAF002210
:0B1EB000AA82AB837402250EFCE4350F
:0B1EBB000FFDC002C003C004C00512F0
:0E1EC60053B1E5828583F0D005D004D003D05F
:0C1ED400022AFAEB35F0FB0ABA00010B01
:0E1EE0008C828D83EAF0A3EBF0EA4B700E8546
:0A1EEE000E82850F83A3A37401F098
:031EF800A3E4F070
:011EFB0022C4
:0A1EFC00850E82850F83A3A3E4F096
:031F0600A3F02223
:071F0900121EB090F2EE126F
:051F10001E39021EFC59
:071F1500C2AF150DAA107503
:021F1C0010FFB4
:0A1F1E00C3EA950D5029EA2A24CEEB
:0B1F2800FBE434F2FCEA04FD25E02499
:0A1F3300CEF582E434F2F583E0FEFF
:0E1F3D00A3E0FF8B828C83EEF0A3EFF08D0209
:021F4B0080D143
:061F4D00E4F50EF50F02A1
:021F53001D0768
:021F55007A0010
:0A1F5700C3EA950D504FEA2A24CE8C
:0C1F6100F582E434F2F583E0FBA3E0FC21
:0E1F6D008B828C83E0FDA3E0FE74062BF582D0
:0E1F7B00E43CF583E0FBA3E0FC7F80C002C0E5
:0C1F890005C006C003C004C007740EC0F1
:0C1F9500E0747AC0E07480C0E0126CDAE6
:0B1FA100E58124F8F581D0020A80AB36
:011FAC002212
:071FAD007510FFE4F50EF5CD
:041FB4000F021D07F4
:0E7A0E00253132733A20776368616E2025308F
:047A1C0034780A00B0
:071FB8001226047811E4F287
:0C1FBF0012251EE58260F97811C3E2F5DE
:0C1FCB00F0740795F040ED7811E275F01D
:061FD70003A4901FDD735E
:071FDD00021FF50223D402EC
:061FE40020E602216D025F
:061FEA0021E002220402C6
:051FF00022E902233884
:0E1FF50090F1B7E0FAA3E0FB4A7003022087E8
:0E20030090F1C4E0FCA3E0FD4C7003022087C6
:0C201100C004C0057827E2FE08E2A2E748
:0E201D0013CE13CEA2E713CE13CEFFEAC39E5E
:0C202B00FCEB9FFD7825C3E29C08E264FA
:0E203700808DF063F08095F0D005D00440421B
:0C204500EE2CFCEF3DFD7825C3E2F5F029
:0E205100EC95F008E2F5F0ED648063F0809508
:0C205F00F040257823C3E2941808E264E6
:0C206B0080947C40177823C3E2F5F074E9
:0E2077005895F008E2F5F0749B63F08095F048
:02208500500AFF
:0A20870078117409F2124B7B8047B8
:0C2091007816E27034EE2AFAEF3BFB7880
:0C209D0025C3E29A08E264808BF063F037
:0B20A9008095F0501C78117402F212B8
:0C20B40059B0758201123CED90006412DE
:0A20C0003C2C75820112491A800EB3
:0C20CA0078117401F2124B7B7582011238
:0220D600491AA5
:0C20D8007A117BFF8A828B83121E770234
:0220E4001FBF1C
:0C20E6007844C3E2F5F0741495F008E2B1
:0C20F200F5F0748063F08095F0403478C5
:0C20FE0048C3E2F5F0744095F008E2F5EC
:0D210A00F0748163F08095F04003021FBF68
:0C2117007846C3E2F5F0745095F008E241
:0E212300F5F0748063F08095F04003021FBF5A
:0A21310078117403F27817E2FA083F
:0C213B00E2FB7812EAF208EBF2122F63CC
:0D21470090000A123C2C758200123CED90B5
:09215400FAA27403F090FAA21241
:0B215D001E777A117BFF8A828B8312B1
:052168001E77021FBFFD
:0C216D007848C3E294D808E26480947FB4
:0C21790050177844C3E2F5F0746495F050
:0D21850008E2F5F0748063F08095F04027CB
:0A21920078177912E3F5F0C3E29527
:0E219C00F0FA09E3F5F008E295F0FBC374DCFD
:0D21AA009A74858BF063F08095F04003027D
:0221B7001FBF48
:0921B90078117404F27848E2F593
:0621C2001808E2F519788F
:0B21C80014E22401F208E23400F27A75
:0B21D300117BFF8A828B83121E7702B3
:0221DE001FBF21
:0C21E0007846C3E2948008E26480948C8E
:0521EC00400302226F18
:0A21F10078117405F27A117BFF8A61
:0921FB00828B83121E77021FBFC4
:0C22040090F1E9E0FAA3E0FB4A603578B5
:0A221000177912E3F5F0C3E295F030
:0C221A00FC09E3F5F008E295F0FD8A6E87
:0C2226008B6F900064C004C005126B3D7B
:0E223200AA82AB83D005D004C3EC9AED9B507A
:0422400003021FBFB7
:0C2244007847E230E72575820012465B07
:0D225000900064123C2C758201123CED7868
:0A225D00117406F27A117BFF8A82E9
:082267008B83121E77021FBFDA
:0A226F00AA18E519A2E7CA33CA3322
:0E227900A2E7CA33CA33CA540330E10244FC60
:0A228700FBE518C39AFAE5199BFB6A
:0C2291007848E2FC08E2A2E7CC33CC3332
:0E229D00A2E7CC33CC33CC540330E10244FC36
:0A22AB00FDEC2AF518ED3BF519C310
:0A22B5007440951874818519F063D8
:0922BF00F08095F04003021FBFFE
:0A22C8007817E2FA08E2FB7812EA48
:0A22D200F208EBF278117403F27ABF
:0B22DC00117BFF8A828B83121E7702A9
:0222E7001FBF17
:0C22E90090F1B5E0FAA3E0FB7844E2FCC1
:0D22F50008E2FDC3EA9CEB9D5003021FBFF1
:0C23020075820112465B7817E224E8F5B2
:08230E001208E23403F51390FC
:0A231600F368E0FAA3E0FB8A168BDF
:04232000178A148B79
:072324001578117407F27A2D
:0B232B00117BFF8A828B83121E770259
:022336001FBFC7
:0C23380090F368E0FAA3E0FBC3EA951400
:0C234400EB64808515F063F08095F0508C
:05235000048A148B1546
:0C23550090F368E0FAA3E0FBC3E5169AE1
:0C236100E51764808BF063F08095F0506D
:05236D00048A168B1725
:0A2372007817E2C39512FA08E2950D
:08237C0013FB30E703021FBF51
:07238400E516C39514FAE50C
:0A238B00179515FBC374049A7480C3
:0C2395008BF063F08095F0401678117416
:0C23A10008F27582001254177A117BFFBD
:0723AD008A828B83121E7768
:0B23B40090F368E0FAA3E0FB8A168BB0
:0423BF00178A148BDA
:0723C300157817E224E8F58C
:0823CA001208E23403F51302CE
:0223D2001FBF2B
:0323D400021FBF26
:0923D7007811E4F27420C0E074F6
:0823E0007AC0E074B8C0E0749B
:0723E8001FC0E090F2EF12AC
:0923EF001C15E58124FCF5812296
:077A2000666C6967687400E1
:0C23F800781FE2FA08E2FBE23395E0FCFB
:0C240400FD7834E22AF208E23BF208E224
:0C2410003CF208E23DF27819E2FA08E222
:0C241C00FBE23395E0FCFD7830E22AF290
:0D24280008E23BF208E23CF208E23DF278E7
:0B2435002EE22401F208E23400F22243
:0C2440007837E23395E0E2A2E71318E2DF
:0C244C0013FB18E2137825F208EBF2787D
:0A24580034E4F208F208F208F2780A
:0C24620033E23395E0E2A2E71318E21326
:0C246E00FB18E213FA7821F208EBF28A66
:0C247A00828B83121264E5828583F07867
:0A24860023F208E5F0F27830E4F2EA
:0C24900008F208F208F2782EE4F208F2DC
:01249C00221D
:0C249D00782EC308E2940250030223F8DA
:0E24A90090F1C4E0FAA3E0FB90F1B7E0FCA3D1
:0C24B700E0FDEAC39CFAEB9DFB7827EAED
:0A24C300F208EBF28A6EEBF56F33BE
:0A24CD0095E0F570F57190D01475DC
:0E24D700F0397401126C15AA82AB83ACF0FDD3
:0C24E5007829EAF208EBF208ECF208EDAE
:0924F100F2122440782DE4F222DD
:0C24FA00782EC308E2940250030223F87D
:0A250600782EC308E29404500C780C
:0B2510002EE22401F208E23400F22267
:03251B0002244057
:0C251E007A1A7BFF8A828B83121E777A68
:0A252A001C7BFF8A828B83121E398E
:06253400E51CB51A0302CC
:02253A0025F981
:0A253C00E51A75F00EA42409FA74E4
:0C254600F535F0FB8A828B83E0FCA3E0FB
:0C255200FD7817ECF208EDF274022AFC90
:0E255E00E43BFD8C828D83A3A3E0FCA3E0FD93
:0C256C007819ECF208EDF28C828D83C02F
:0E25780002C003121264AC82AD83D003D00205
:0A258600781BECF208EDF27823D385
:0C259000E29CF4B3FCB308E29DF4FD787B
:0C259C001DECF208EDF274022AFAE43B98
:0C25A800FB8A828B83E0FCA3E0FD781F1F
:0C25B400ECF208EDF290F1CFE0600C7842
:0B25C0001F74FFC39CF2747F9D08F2A3
:0C25CB008A828B83781FE2F0A308E2F004
:0A25D700782DE2600512249D800EAD
:0625E1007811E2B40300D2
:0525E70050031224FA6C
:0325EC00122A5F51
:0825EF00E51A04541FF51A025D
:0225F700253489
:0625F900782DE2B40100A0
:0525FF00E433F5822227
:0A260400120AC2782EE4F208F27800
:0A260E0030E4F208F208F208F27856
:0A26180019E4F208F27834E4F20845
:0C262200F208F208F2781FE4F208F285DA
:03262E001C1A78FB
:052631002D7401F222EE
:082636007846E2F56E08E2F5BA
:08263E006FE23395E0F570F541
:0C2646007190028FE4F5F0126BA7858202
:062652002385832485F0BE
:0426580025F52678C6
:07265C0048E2F52708E2F552
:0826630028E23395E0F529F5AA
:03266B002A852796
:03266E006E85284E
:032671006F852949
:0326740070852A44
:0C26770071900003E4F5F0126BA7AC8238
:0B268300AD83AAF0FBEC2523FCED3535
:08268E0024FDEA3525FAEB35C5
:0C26960026FBEDC4CCC4540F6CCC540FD8
:0E26A200CC6CCCFDEAC454F04DFDEBC4CAC4B0
:0E26B000540F6ACA540FCA6ACA30E30244F0DB
:0C26BE00FB7838E22CF208E23DF208E262
:0A26CA003AF208E23BF285276E8524
:0326D400286F85E7
:0326D700297085E2
:0926DA002A7190028FE4F5F01260
:0C26E3006BA7AA82AB83ACF0FD783CE250
:0E26EF002AF208E23BF208E23CF208E23DF279
:0126FD0022BA
:0A26FE00783AE2FA08E2FB781DE2E8
:0C270800C39AFA08E29BFB784EEAF20844
:0D271400EBF2EB30E707C3E49AFAE49BFB1D
:0E272100C3747F9A74808BF063F08095F05043
:05272F00047A7F7B002D
:0C2734007850E2FC08E2A2E713CC13CCC2
:0C274000A2E713CC13CCFD7850E2C39C40
:0A274C00F208E29DF28A6E8B6F8A9C
:0E275600828B83126B3DAA82E583A2E713CA31
:0C27640013CAA2E713CA13CAFB7850E2A4
:0C2770002AF208E23BF27811E2B4060005
:03277C00400122F7
:0C277F00781BE22420FA08E234D1FB7839
:0C278B0046E22480FC08E234F3FDC42385
:0E279700CCC423541F6CCC541FCC6CCC30E44B
:0327A5000244E00B
:0E27A800FDC3E49C74808DF063F08095F050CA
:0E27B60013C3EA9CEB64808DF063F08095F015
:0627C40050048C028D039D
:0E27CA00C3E49A74808BF063F08095F0504B5E
:0E27D800C3E49A74818BF063F08095F0500496
:0427E6007A007B01F9
:0C27EA00784EE2FC08E2FDE23395E0FED0
:0C27F600FFE4C39AFA74019BFB8A6EEBAF
:08280200F56F3395E0F570F568
:0C280A00718C828D838EF0EF126BA7AAF8
:0C28160082AB83ACF0FD784EEBF208ECD6
:01282200F2C3
:012823002292
:072824001226FE784EE2F5DA
:0A282B002B08E2F52CE23395E0F5EE
:042835002DF52E85CA
:032839002B6E857E
:03283C002C6F8579
:03283F002D708574
:092842002E71900789E4F5F012F3
:0C284B006BA7AE82AF83AAF0FB7838E2E6
:0E2857002EF208E23FF208E23AF208E23BF20B
:04286500852B6E85CC
:032869002C6F854C
:03286C002D708547
:09286F002E7190B40FE4F5F01293
:0C2878006BA7AA82AB83ACF0FD783CE2B9
:0E2884002AF208E23BF208E23CF208E23DF2E2
:04289200852B6E859F
:032896002C6F851F
:032899002D70851A
:09289C002E71908682E4F5F01221
:0C28A5006BA7AA82AB83ACF0FD7840E288
:0E28B1002AF208E23BF208E23CF208E23DF2B5
:0128BF0022F6
:0C28C00090F1B7E0FAA3E0FB781FD3E230
:0E28CC009AF4B3FAB308E29BF4FB3395E0FCF8
:0928DA00FD7829E2F56E08E2F533
:0828E3006F08E2F57008E2F550
:0C28EB00718A828B838CF0ED126BA7AA1F
:0C28F70082AB83ACF0FD7840D3E29AF491
:0E290300B3B308E29BF4B3B308E29CF4B3FC58
:0C291100B308E29DF4FD7852ECF208EDF2
:02291D00F222A4
:07291F001226FE1228C07809
:072926004EE2F52F08E2F577
:08292D0030E23395E0F531F5CD
:0329350032852FB9
:032938006E853079
:03293B006F853174
:03293E007085326F
:0C2941007190028BE4F5F0126BA7858208
:06294D003385833485F0A0
:0429530035F53678A8
:0729570052E2F53708E2F53A
:08295E0038E23395E0F539F58C
:032966003A853778
:032969006E853840
:03296C006F85393B
:03296F0070853A36
:0C29720071900005E4F5F0126BA7AE8236
:0B297E00AF83AAF0FBEE2533FEEF351F
:0829890034FFEA3535FAEB35A5
:0A29910036FB7838E22EF208E23F30
:0B299B00F208E23AF208E23BF2852F5E
:0329A6006E85300B
:0329A9006F853106
:0329AC0070853201
:0C29AF0071901460E4F5F0126BA78582B3
:0629BB003385833485F032
:0429C10035F536852D
:0329C500376E85E5
:0329C800386F85E0
:0329CB00397085DB
:0929CE003A71900274E4F5F01274
:0C29D7006BA7AE82AF83AAF0FBEE2533A5
:0A29E300FEEF3534FFEA3535FAEB5C
:0A29ED003536FB783CE22EF208E2DA
:0C29F7003FF208E23AF208E23BF2852FC2
:032A03006E8530AD
:032A06006F8531A8
:032A0900708532A3
:0C2A0C007190014AE4F5F0126BA785827E
:062A18003385833485F0D4
:042A1E0035F53685CF
:032A2200376E8587
:032A2500386F8582
:032A28003970857D
:092A2B003A71901082E4F5F012FA
:0C2A34006BA7AE82AF83AAF0FBEE253347
:0A2A4000FEEF3534FFEA3535FAEBFE
:0A2A4A003536FB7840E22EF208E278
:0B2A54003FF208E23AF208E23BF222F7
:0C2A5F001226367811C3E2F5F0740595DC
:082A6B00F0400512291F800351
:032A730012282402
:0A2A7600783AE2FA08E2FB7844EA3D
:0A2A8000F208EBF2783C79460808F2
:0A2A8A00E2F308E209F3784079480E
:0E2A94000808E2F308E209F390F366E0FCA301
:0C2AA200E0FD7844C3E2F5F0EC95F0088C
:0E2AAE00E2F5F0ED648063F08095F050089042
:072ABC00F366EAF0A3EBF062
:0E2AC30090F368E0FAA3E0FB3395E0FCFD78A9
:0A2AD1004AE2C39AF53B08E29BF5C8
:0A2ADB003C08E29CF53D08E29DF581
:0A2AE5003E781DE2FE08E2FFE23336
:0A2AEF0095E0FAFBEE253BFEEF3503
:082AF9003CFFEA353DFAEB3524
:0A2B01003EFB784AEEF208EFF208FE
:0C2B0B00EAF208EBF2784AE2243FFA08F4
:0E2B1700E23400FB08E23400FC08E23400FD6A
:0E2B2500EBA2E7CA33CA33CA5401FBEC2C4BB7
:0E2B3300FBEDA2E7CC33CC33CC540130E002F2
:022B410044FE50
:092B430090F368EAF0A3EBF02224
:032B4C00026927F4
:0E2B4F00E58275F003A42480FAE435F0FB3330
:0A2B5D0095E0FC8A828B838CF02245
:0E2B6700AA8290F36EE4F090F36CE0FBA3E022
:0E2B7500FC90F36FEBF0A3ECF08A82122B4F72
:0C2B8300AA82AB83ACF0FD78E4E22AFAF1
:0E2B8F0008E23BFB08E23CFC08E23DFD74035B
:0A2B9D00C0E0E4C0E0746EC0E07414
:0B2BA700F3C0E08A828B838CF0ED12FB
:0B2BB2001946E58124FCF5810269272B
:0C2BBD00122B4FAA82AB83ACF0FD78E431
:0E2BC900E22AFA08E23BFB08E23CFC08E23D8F
:0C2BD700FD7403C0E0E4C0E0746EC0E0D8
:0C2BE30074F3C0E08A828B838CF0ED124A
:092BEF00182DE58124FCF581227A
:042BF8007A007B00E4
:032BFC00BB10000B
:0E2BFF00503A8B82C002C003122BBDD003D00F
:0E2C0D000290F36EE0FC701990F36FE0FDA3EF
:0E2C1B00E0FE90F36CE0FFA3E0F8EDB50705D6
:052C2900EEB5000122E0
:082C2E00EC60058A82022B67AD
:052C36000B8B0280C1C0
:032C3B000208E9A3
:092C3E0090F1CAE0F56EA3E0F587
:082C47006FA3E0F570A3E0F5B6
:0A2C4F007178E4E2F58208E2F583F3
:092C590008E2F5F008E2026AD875
:0B2C6200AA8290F1CAE0F56EA3E0F535
:082C6D006FA3E0F570A3E0F590
:0C2C7500717B007C007D008A828B838CC8
:052C8100F0ED026BA75D
:0E2C86007A007B00C002C003122C3EAC82D04C
:052C940003D0027D00E9
:0E2C9900C3ED9C503D8D82C002C003C004C03C
:0E2CA700051234EDAE82AF83D005D004D00309
:0E2CB500D002EE4F601DEA4B6015EEC39AF898
:0E2CC300EF9BF9C3E498748089F063F080956C
:032CD100F05004BC
:042CD4008E028F03DA
:032CD8000D80BEAE
:052CDB008A828B8322B8
:0A2CE000C04CE581F54C2404F58199
:0E2CEA00AA82C002122BF8D0028A82122C623B
:0C2CF800AA82AB83ACF0FDA84C08A60239
:0E2D040008A60308A60408A60590F1CAE0FE82
:0C2D1200A3E0FFA3E0FAA3E0FBA84C083C
:0E2D1E00EE26FEEF0836FFEA0836FAEB08361E
:052D2C00FB8E048F0581
:0C2D3100A84C08C3E69C08E69D08E69A42
:082D3D0008E69B4003022DF49F
:022D45007E000E
:032D4700BE1000BB
:0E2D4A005069C004C005C002C0038E077A00A5
:0C2D58007B007C00A84C08EF26FFEA0876
:0E2D640036FAEB0836FBEC0836FCC003C00460
:0C2D7200C005C0067401C0E0E4C0E074BD
:0A2D7E0071C0E074F3C0E08F828A98
:0E2D8800838BF0EC12182DAA82E58124FCF555
:0E2D960081D006D005D004D003EAD003D002CD
:0E2DA400D005D004600890F371E0FFBFFF037C
:032DB2000E8092FE
:052DB500BE1002803A8F
:0C2DBA00A84C0886820886830886F00872
:0E2DC600E6C002C003C004C005126936D00585
:0A2DD400D004D003D002A84C087907
:0C2DDE00E0E326F609E30836F609E308F6
:0A2DEA0036F609E30836F6022D3133
:062DF400854C81D04C2249
:022DFA007A104D
:0E2DFC008A031AEB60478A82C002122BBDD0F8
:0E2E0A000290F36EE070EB90F36CE0FAA3E040
:0E2E1800FB4A601D90F36FE0FCA3E0FDECC3ED
:0E2E26009AFAED9BFBC3E49A74808BF063F084
:052E34008095F0501034
:0E2E390090F36FE0FAA3E0FB90F36CEAF0A3D5
:022E4700EBF0AE
:0E2E490090F36CE0FAA3E0FB4A700990F36C82
:062E57007401F0E4A3F099
:012E5D002252
:0A2E5E00C04CE581F54C2404F58119
:0B2E6800120AC2122C86AA82AB8390D3
:0E2E7300F36CEAF0A3EBF0EA4B601A0ABA0027
:022E8100010B43
:0D2E830090F36CEAF0A3EBF0EA4B700990BD
:082E9000F36C7401F0E4A3F0FF
:0C2E9800122DFA7858E4F208F208F20853
:0C2EA400F27854E4F208F208F208F2128E
:0E2EB0002C3EAA8290F36CE0FBA3E0FC1BBB5F
:032EBE00FF011CF5
:0A2EC1008A6E756F008B828C83C04F
:0A2ECB0002126B5AAB82D0028B0496
:0E2ED5008C82C002C003C0041234EDE5828579
:0E2EE30083F0D004D003D00245F070548C82EE
:0C2EF100122C62AA82AB83ACF0FD785476
:0E2EFD00EAF208EBF208ECF208EDF290F1CAEE
:0C2F0B00A84C08E0F6A3E008F6A3E008DC
:0C2F1700F6A3E008F6A84C08E62AF6082D
:0C2F2300E63BF608E63CF608E63DF6A8A2
:0A2F2F004C087958E6F30809E6F3B0
:0A2F39000809E6F30809E6F3801129
:082F43000CC3EC9A40027C0073
:062F4B00ECB50302800357
:032F5100022ED578
:0A2F540090F36C121E777582008561
:052F5E004C81D04C2263
:0A2F630090F36B7401F090F36B0221
:022F6D001E77CD
:082F6F0090F36BE4F0022B4C1F
:0E2F7700122C86AA82AB83E4BA0004BB0001D0
:012F85000447
:042F8600FAB4010098
:052F8A00E433F5822292
:0A2F8F0078547958E2F5F0E3B5F04C
:0E2F99001F08E2F5F009E3B5F01608E2F5F0C6
:0E2FA70009E3B5F00D08E2F5F009E3B5F0041A
:042FB5007401800122
:012FB900E433
:032FBA00F582227B
:0A2FBD00C04C85814C05810581059B
:0B2FC70081122C3EAA82A84C08760064
:0B2FD200A84C08C3E69A4003023060E0
:0C2FDD00A84C088682C0021234EDAC82C1
:0C2FE900AD83D002A84C0808A60408A67E
:0C2FF50005A84C0808E60846605AC00217
:0C300100A84C08E604F582122C62AF8394
:0C300D00AAF08F068A07A84C088682C033
:0E30190006C007122C62AC83ADF0D007D006C3
:0E3027008C028D04C002C006C007C002C004A7
:0C303500A84C0808E6C0E008E6C0E07403
:0A30410027C0E0747AC0E07480C07C
:0E304B00E0126CDAE58124F7F581D002D002A4
:07305900A84C0806022FD26B
:0A3060007442C0E0747AC0E074808E
:0C306A00C0E0126CDA158115811581851B
:053076004C81D04C224A
:09307B001204AC7807E2600122A6
:0C308400122C3EAA827800E2F5F008E26F
:0830900045F060407B007C006C
:0E309800C3EC9A50378C82C002C003C00412F1
:0D30A60034EDAD82AE83D004D003D00278AB
:0C30B30000E2B5050708E2B50602800245
:0230BF00800E81
:0C30C1008B82122CE0907A4875F080029F
:0230CD006C672E
:0530CF000C8C0380C41D
:0A30D4007800E2C0E008E2C0E074FA
:0A30DE004FC0E0747AC0E07480C0B7
:0B30E800E0126CDAE58124FBF5812288
:0B30F30090F36BE4F078607409F29039
:0630FE007A6312077374EF
:083104006FC0E0747AC0E074B2
:08310C001FC0E07432C0E09026
:0C311400F372121C15E58124FCF58122E9
:0E7A2700666C69676874202564207374617250
:0D7A35007420257820656E642025780A00F5
:067A4200646F6E650A008E
:077A480045726173656400E3
:0E7A4F004E6F207375636820666C69676874FB
:067A5D003A2025640A0036
:027A6300BD2F35
:027A6500737A32
:027A67007B3072
:067A69007F7A000000001E
:047A6F006C6F6700D1
:0C7A73006C004C697374206C6F6773002A
:0E7A7F0064203C666C696768742D6E756D62DC
:0E7A8D0065723E0044656C65746520666C6928
:047A9B0067687400A4
:08312000AA82AB837C5A7D00FA
:03312800BD0800DF
:0E312B0050118A828B83E0FEA3AA82AB83EE52
:053139002CFC0D80EAF2
:06313E00C3E49CF58222AF
:0E314400AA82AB837C0074012AFDE43BFE8D61
:0E315200828E83E4F08A828B83C002C003C0A9
:0E31600004C005C006123120AF82D006D00593
:0E316E008D828E83EFF090F36A121534D00438
:0A317C00D003D00278547958C3E361
:0E318600F5F0E295F009E3F5F008E295F009A6
:0E319400E3F5F008E295F009E3F5F008E295A6
:0E31A200F0401690F36BE0FD600FC002C0031A
:0B31B000C004122F6FD004D003D00227
:0E31BB0090F36BE0FD603E7C01C0047408C020
:0C31C900E0E4C0E0C002C0037854E2F56E
:0E31D5008208E2F58308E2F5F008E2121946DE
:0C31E300E58124FCF581D0047854E2243E
:0E31EF0008F208E23400F208E23400F208E2CE
:0331FD003400F2A9
:0D32000090F36AC004121592D0048C822253
:0E320D0090F3E9123120E58260047582002200
:04321B007582012295
:06321F00126535122E5E5F
:0B32250090F36BE0FA700890F36B125E
:043230001E3980F1D2
:0A32340090F3E97446F090F3EB7894
:0B323E0017E2F0A308E2F090F3ED7837
:0C32490025E2F0A308E2F090F36CE0FA3C
:0E325500A3E0FB90F3EFEAF0A3EBF090F3E9B7
:09326300123144E51A04541FF570
:0A326C001B75F00EA42409F582740E
:0C327600F535F0F583E0FAA3E0FB8A04D4
:063282008B057860E4F208
:06328800E51AB51B03026C
:02328E003450BA
:0C329000C002C003E51B75F00EA4FEAFE9
:0A329C00F02409F582EF34F5F58304
:0E32A600E0FAA3E0FB90F3EBEAF0A3EBF0906C
:0E32B400F3EBE0FAA3E0FBEAC39CEB9DD00332
:0832C200D00230E70302334F94
:0C32CA00C002C00390F3E97441F0EE2450
:0A32D60009FAEF34F5FB8A828B83BE
:0E32E000A3A3E0FAA3E0FB90F3EDEAF0A3EB6A
:0A32EE00F0EE2409FEEF34F5FF7442
:0E32F800022EFEE43FFF8E828F83A3A3E0FA36
:0E330600A3E0FB90F3EFEAF0A3EBF090F3E905
:0C331400C002C003123144D003D0027884
:0C33200060C3E2F5F0740595F0D003D016
:0E332C0002401190F3EBE0FEA3E0FF74012ECF
:06333A00FCE43FFD800FE2
:0E33400090F3EBE0FEA3E0FF740A2EFCE43FE6
:01334E00FD81
:0E334F0090F3EBE0FEA3E0FFEEC39AFEEF9BCF
:07335D00FF30E703023446D4
:0C336400C004C00590F3E97454F0E51BB0
:0C33700075F00EA4FEAFF02409FCEF3451
:0C337C00F5FD74022CFCE43DFD8C828DFC
:0E33880083A3A3A3A3E0FCA3E0FD90F3EDEC70
:0A339600F0A3EDF0EE2409FEEF3481
:0C33A000F5FF74022EFEE43FFF74062EC1
:0E33AC00F582E43FF583E0FCA3E0FD90F3EF33
:0D33BA00ECF0A3EDF090F3E9C004C00512A3
:0D33C7003144D005D00490F3E97444F0E5E2
:0A33D4001B75F00EA4FCADF02409F7
:0C33DE00FEED34F5FF74022EFEE43FFF0C
:0E33EA0074082EF582E43FF583E0FEA3E0FFB9
:0C33F80090F3EDEEF0A3EFF0EC2409FCE4
:0C340400ED34F5FD74022CFCE43DFD7479
:0E3410000A2CF582E43DF583E0FCA3E0FD907C
:0E341E00F3EFECF0A3EDF090F3E9C004C0056D
:0E342C00123144D005D00490F3EBE0FCA3E095
:0C343A00FD74202CFAE43DFBD005D0040A
:08344600E51B04541FF51B02F5
:02344E003288C2
:0A34500078117960E2F5F0E3B5F0C1
:03345A0002805895
:08345D007811E2FE7860F290A4
:09346500F3E97453F090F3EB78E5
:0C346E0017E2F0A308E2F07F0090F3EDFD
:0D347A00EEF0A3EFF090F3EFE4F0A3F0907C
:0E348700F3E9C002C003C004C005123144D0F6
:0C34950005D004D003D0027860E2B40837
:0E34A10013C002C003C004C005122F6FD00577
:0634AF00D004D003D0029E
:0E34B50090000AC002C003C004C005121F0927
:0834C300D005D004D003D002B3
:0A34CB0090F36BE0FE60030232880C
:0E34D50090F36BC002C003C004C005121E3984
:0A34E300D005D004D003D00280DE33
:0E34ED00122C62AA82AB83ACF0FD7408C0E022
:0A34FB00E4C0E074E9C0E074F3C01F
:0E350500E08A828B838CF0ED12182DAA82E5ED
:0C3513008124FCF581EA70049000002285
:0E351F0012320DE582601590F3E9E0FABA462B
:0E352D000D90F3EFE0FAA3E0FB8A828B83227D
:04353B0090000022DA
:017A9F0001E5
:0C353F007811E2907AA093FA74075AFB0E
:04354B00EA700122FF
:0E354F008B041BEC604CEA30E31BC002C0038F
:0E355D007414C0E0E4C0E075825E12402C15CC
:09356B00811581D003D002801902
:0E357400C002C0037406C0E0E4C0E075825ED1
:0B35820012402C15811581D003D002EF
:0E358D00900006C002C003121F09D003D00236
:06359B00EAC313FA80AE42
:0635A100900024021F0946
:0E35A700E582FA70197432C0E0E4C0E075826B
:0E35B5005E12402C15811581900014121F0922
:0235C300802363
:0E35C5008A031AEB601DC0027414C0E0E4C05B
:0E35D300E075825E12402C1581158190001467
:0735E100121F09D00280DD7A
:0635E80090001E021F0905
:0C35EE00AA82E583FB30E7047A007B0032
:0235FA007C0053
:0A35FC008C050CED24F1FDE434F31E
:0A360600FE756E0AE4F56F8A828BF0
:0E36100083C002C003C004C005C0061272BC15
:0E361E00AF82D006D005D004D003D0028D823A
:0A362C008E83EFF0756E0AE4F56F6F
:0E3636008A828B83C0041272F2AA82AB83D008
:0736440004EA4B70B38C0295
:0A364B001AEA24F1F582E434F3F5E5
:0E36550083E0F582C0021235A7D002EA70E8C9
:013663002244
:0D36640090F366E0FAA3E0FB8A828B8302FC
:0236710035EE34
:0C367300124679AA82BA01047A01800292
:02367F007A00CF
:033681008A822218
:0E368400758200123673AA82758201C002128E
:0C3692003673AB82D002EB2B4AF582228B
:08369E00123684E582FA602374
:0E36A6008A031AEB604DC0027402C0E0E4C05B
:0E36B400E075824B12402C1581158190000AA2
:0736C200121F09D00280DD98
:0236C9007A0580
:0E36CB008A031AEB6028C0027402C0E0E4C05B
:0E36D900E075824B12402C158115817402C0E1
:0E36E700E0E4C0E075829612402C158115813A
:0436F500D00280D2AD
:0E36F900122F8FE582605890000A121F097A86
:0137070002BF
:0E3708008A031AEB604AC002740AC0E0E4C0F3
:0E371600E075829612402C15811581740AC050
:0E372400E0E4C0E075825E12402C1581158134
:0E373200740AC0E0E4C0E075824B12402C1512
:0E374000811581740AC0E0E4C0E075825E125B
:0A374E00402C15811581D00280B0D7
:01375800224E
:073759007811E27861F21221
:09376000353F7861E2B4080B1258
:0A37690036649001F4121F0980E697
:093773007861E2B4010312369EF4
:0B377C007811E2B4021D12369E7A3272
:0C3787008A031AEB60EF7811E2B402E94B
:0C37930090000AC002121F09D00280E85A
:0A379F0078617911E2F5F0E3B5F06E
:0C37A900AF7A117BFF8A828B83121E39DD
:0237B50080E8AA
:0937B70074AAC0E0747AC0E07449
:0837C00059C0E07437C0E0902D
:0C37C800F3FB121C15E58124FCF58122A6
:0A7AA0000302340C242C0B1A144CC2
:077AAA007265706F72740039
:0401B8007864E4F291
:0A37D400E51A14541F75F00EA4242A
:0A37DE0009FA74F535F0FB8A828BBE
:0E37E80083E0FCA3E0FD90F474ECF0A3EDF0A0
:0A37F60090F4767401F090F47778F7
:0C38000011E2F08A828B83A3A3E0FCA3FA
:0E380C00E0FD90F478ECF0A3EDF074022AFADF
:0E381A00E43BFB8A828B83A3A3E0FCA3E0FDCA
:0E38280090F47AECF0A3EDF08A828B83A3A3D8
:0E383600A3A3E0FCA3E0FD90F47CECF0A3ED76
:0E384400F074062AF582E43BF583E0FCA3E075
:0E385200FD90F47EECF0A3EDF074082AF582F0
:0E386000E43BF583E0FCA3E0FD90F480ECF087
:0E386E00A3EDF0740A2AF582E43BF583E0FA3C
:0E387C00A3E0FB90F482EAF0A3EBF090F4845A
:0C388A007848E2F0A308E2F090F48678A1
:0B38960046E2F0A308E2F090F488780E
:0B38A10044E2F0A308E2F090F48A7803
:0B38AC0021E2F0A308E2F090F48C7819
:0C38B70025E2F0A308E2F090F1B7E0FA7F
:0E38C300A3E0FB90F48EEAF0A3EBF090F1C4CA
:0E38D100E0FAA3E0FB90F490EAF0A3EBF074B1
:0C38DF0020C0E090F472124CBF15812252
:0A38EB007868E214F27868C3E2F591
:0B38F500F0748063F08095F050012219
:0D39000090F4767404F090F477740BF012DC
:0C390D002F8FE58260067A007B008008A6
:0839190090F36CE0FAA3E0FB5F
:0E39210090F478EAF0A3EBF090F47A7401F0E1
:0E392F0090F47B7415F090F1C3E0FA7B0090E9
:0E393D00F47CEAF0A3EBF090F1B5E0FAA3E021
:0E394B00FB90F47EEAF0A3EBF090F1CAE0A34B
:0E395900E0FBA3E0FCA3E0FD8B02ECC313CA6D
:0E39670013CAC313CA13CAFBED030354C04BAB
:0E397500FBED0303543F90F480EAF0A3EBF067
:08398300740724B3F56EE4346F
:04398B00F1F56F756E
:06398F007008E4F57190E0
:06399500F4821251E27AF7
:04399B00B77B7F8AED
:04399F006E8B6F7547
:0639A3007008E4F57190CC
:0A39A900F48A1251E27420C0E0908D
:0839B300F472124CBF1581787B
:0639BB0067E27868F222C9
:0A39C100786AE214F2786AC3E2F5B6
:0E39CB00F0748063F08095F0404790F47674BD
:0B39D90005F090FAA3121534740524C9
:0539E400A4F56EE434BF
:0439E900FAF56F7507
:0639ED00701BE4F571906F
:0639F300F4771251E2908E
:0B39F900F4747892E2F0A308E2F09072
:0A3A0400FAA31215927420C0E0909E
:083A0E00F472124CBF1581781F
:063A160069E2FA786AF291
:013A1C002287
:0A3A1D00786BE214F2786BC3E2F557
:0E3A2700F0748063F08095F0404490F4767463
:093A350006F090FAA3121534907A
:0A3A3E00FAC9E090F477F074062452
:053A4800C4F56EE4343A
:043A4D00FAF56F75A2
:063A51007018E4F571900D
:063A5700F4781251E29028
:0A3A5D00FAA31215927420C0E09045
:083A6700F472124CBF158178C6
:063A6F0069E2FA786BF237
:013A7500222E
:0A3A7600786DE214F2786DC3E2F5FA
:0E3A8000F0748063F08095F0405A90F47674F4
:0E3A8E0007F090FA0CE0FAA3E090F477EAF06B
:093A9C0090FA10E090F478F0902B
:083AA500FA11E090F479F090B1
:063AAD00FA2A121534751F
:033AB3006E12751B
:033AB6006FFA9014
:0B3AB900FA11E075F002A4F57085F032
:053AC4007190F47A127C
:063AC90051E290FA2A12FE
:0A3ACF0015927420C0E090F472120A
:093AD9004CBF1581786CE2FA780B
:023AE2006DF283
:013AE40022BF
:0A3AE500120AC290F1D4E07003123F
:023AEF001F15A1
:0E3AF10090F36CE0FAA3E0FB4A700890F36CCF
:053AFF00121E3980EDEC
:0E3B04009000A4E493FA740193FB90F472EA2B
:043B1200F0A3EBF041
:0C3B16007862E2F5F008E245F0700890DB
:073B2200F472121E3980ED60
:0C3B29001253B1AA82AB837865EAF2085F
:023B3500EBF2B1
:0C3B37007862E2F5F008E245F060D4127C
:0A3B430053B11253B1AC82AD837888
:0C3B4D0062E22CFA08E23DFBC002C0035B
:0C3B59001237D4D003D0027891E2600B48
:0B3B6500C002C003123A76D003D00269
:0B3B7000C002C0031239C1123A1D123E
:0C3B7B0038EBD003D0027864E2606CC02C
:0E3B870002C0031253B1AC82AD83D003D00252
:0C3B95007865D3E29CF4B3FCB308E29D19
:0E3BA100F4FD20E74CC002C0031253B1E582D0
:0C3BAF008583F0D003D002786524F4F286
:0C3BBB00740135F008F27811E2B4022029
:0E3BC700C002C003123684AC82D003D002ECE0
:0E3BD500FD600F8D82C002C003124EA4D0030B
:043BE300D002800B81
:0B3BE700C002C003124E7AD003D002CF
:0E3BF200C002C0031253B1AC82AD83D003D029
:0E3C000002EAC39CFAEB9DFBC3E49A74808B2E
:0B3C0E00F063F08095F04003023B37AC
:0B3C19008A828B83121EB090F472129E
:063C24001E39121EFC0215
:023C2A003B3726
:0C3C2C00AA82AB837C007862EAF208EB0D
:0D3C3800F290FA10E0700690FA107464F03B
:0A3C450090FA10E0FD7E008A6E8BFD
:0C3C4F006F8D828E83C002C003C004127F
:0D3C5B006AAFAD82AE83D004D003D00278F2
:0C3C68006CEDF2C374808DF063F0809569
:053C7400F050027C018C
:073C7900786DECF28A6E8BFE
:0B3C80006F900064C002C003C004127B
:0D3C8B006AAFAD82AE83D004D003D00278C2
:0C3C980069EDF2C3EC64808DF063F080F5
:053CA40095F050010C39
:0C3CA900786AECF2C3EC64808DF063F0EC
:063CB5008095F050010CA7
:073CBB00786BECF28A6E8BBE
:0C3CC2006F9001F4C004126AAFAA82AB3C
:0C3CCE0083D0047867EAF2C3EC64808ABB
:093CDA00F063F08095F050010C3C
:083CE3007868ECF290F4720223
:023CEB001E7742
:0C3CED00AA827864EAF2EA7003024EDF5B
:0C3CF9001253B1E5828583F0786524F455
:083D0500F2740135F008F2220E
:093D0D0074B1C0E0747AC0E074E6
:083D1600E5C0E0743AC0E09042
:0C3D1E00F492121C15E58124FCF58122B2
:0A7AB10074656C656D6574727900F0
:0A3D2A00C04C85814CC082C083C0EC
:0C3D3400F0C0E0786EE4F208F208F2083B
:0A3D4000F27872E4F278737445F231
:0D3D4A000874AFF20874FCF20874FFF2A8D0
:0C3D57004C08E6248AFE08E6345EFF08F3
:0C3D6300E634F9FA08E634FFFBA84C082F
:0E3D6F00A60608A60708A60208A603EB30E782
:0A3D7D001878727401F2A84C08C314
:0E3D8700E496F608E496F608E496F608E4964C
:013D9500F637
:0C3D9600A84C0886020886030886040872
:023DA200860594
:0C3DA4007873C3E2F5F0E495F008E2F556
:0E3DB000F0E495F008E2F5F0E495F008E2F595
:0C3DBE00F0748063F08095F0502C787356
:0E3DCA00E2248AF208E2345EF208E234F9F2F2
:0C3DD80008E234FFF2786EE22401F208E9
:0E3DE400E23400F208E23400F208E23400F2A9
:023DF20080B09F
:0A3DF4007873E54C24FAF9E227F297
:0E3DFE0008E20937F208E20937F208E2093755
:0E3E0C00F21ABAFF091BBBFF051CBCFF011D0B
:073E1A00ED20E703023DA4C7
:0A3E21007872E2601A786EE2D3F4C2
:0E3E2B003400F208E2F43400F208E2F434004D
:073E3900F208E2F43400F28C
:0A3E4000E54C24FAF8796EE326FA47
:0E3E4A0009E30836FB09E30836FC09E30836F5
:0A3E58008A828B838CF0854C81D0A8
:023E62004C22F0
:043E640075B6B0225D
:0A3E6800E51A14541F75F00EA4248F
:043E720009F56E746C
:063E7600F535F0F56F7553
:063E7C00700EE4F5710276
:023E820051E20B
:0C3E8400C022C0E0C0F0C082C083C002B9
:0E3E9000C003C004C005C006C007C000C001CA
:0E3E9E00C0D075D000740F55B5FABA0E027A76
:013EAC000213
:0A3EAD00E51C75F00EA42409FB7457
:0C3EB700F535F0FC74022BFBE43CFC8AA7
:0E3EC30005E4CD25E0CD33FEED2BFBEE3CFCFF
:0E3ED1000A8B828C83E5BAF08B828C83A3E58A
:053EDF00BBF0BA060073
:0A3EE400500FBA020575B63E8005C6
:053EEE0074B04AF5B6B6
:023EF300803815
:0A3EF500E51C75F00EA42409FA7410
:0C3EFF00F535F0FBC002C0031253B1AC5B
:0E3F0B0082AD83D003D0028A828B83ECF0A3B8
:0A3F1900EDF0E51C04541FF51C7ABE
:0A3F23001C7BFF8A828B83121E773D
:0E3F2D00D0D0D001D000D007D006D005D004EF
:0D3F3B00D003D002D083D082D0F0D0E0D0EF
:023F4800223223
:0A3F4A00C04CE581F54C2408F58118
:073F540090F6C9123E6890CF
:0E3F5B00F6D5E0FAA3E0FB90F6D3E0FCA3E07D
:0C3F6900FD90F6D1A84C080808E0F6A373
:0C3F7500E008F690F6CFA84C08E0F6A398
:0C3F8100E008F690F6CDE54C2405F8E0D1
:0C3F8D00F6A3E008F690F6CBE54C240704
:0E3F9900F8E0F6A3E008F690F6C9E0FEA3E01B
:0C3FA700FFC002C003C004C005A84C0805
:0C3FB3000808E6C0E008E6C0E0A84C08E2
:0C3FBF00E6C0E008E6C0E0E54C2405F890
:0C3FCB00E6C0E008E6C0E0E54C2407F882
:0C3FD700E6C0E008E6C0E0C006C00774C9
:0A3FE300BBC0E0747AC0E07480C037
:0C3FED00E0126CDAE58124EFF581854CD0
:043FF90081D04C2205
:0E3FFD0075F23BC28D43A802907B050207734C
:0E7ABB007469636B3A2025357520616363653D
:0E7AC9006C3A2025356420707265733A2025D2
:0E7AD70035642074656D703A20253564206298
:0E7AE5006174743A202535642064726F6775F1
:0E7AF300653A20253564206D61696E3A2025C4
:047B010035640A00DD
:027B05004A3FF5
:067B07000D7B00000000F0
:0E7B0D00610043757272656E7420414443003E
:0E400B00E582FA7009C2A053F5FE75EB0022A3
:0E401900ABF574FE5BF5F0740145F0F5F58A29
:05402700ED75EBB22273
:06402C00C04C85814C121E
:0C403200400BE54C24FCF88682088683D5
:0A403E00121F0975820012400BD01A
:024048004C2208
:0E404A00C2A053F5FEAAF174EF5AF5F07410FF
:0840580045F0F5F175EC1422AE
:0A406000C04C85814CE582FAF4FBA8
:0C406A00E5905203A84C181818E652020A
:09407600EA4BF5900000D04C2249
:0A407F00AA8243902043FE207B0834
:084089007C00EA30E7027C2014
:0E409100EA2AFA74104CFDC002C003C004C03D
:0D409F000575823012406015817582301267
:0E40AC0040601581D003D002DBD353FEDF222B
:0440BA007A007B0805
:0E40BE00EA2AFAC002C0037410C0E075821036
:0E40CC001240601581D003D0023095034302EC
:0140DA0001E4
:0E40DB00C002C003E4C0E07582101240601500
:0A40E90081D003D002DBCE8A8222D0
:0E40F300AA82758255C00212407FD0028A82D6
:0641010012407F0240BAEB
:0A410700C04C85814CAA82758256D7
:0D411100C00212407FD0028A8212407FA8B7
:0A411E004C181818868212407F1218
:0541280040BAD04C225A
:0A412D00C04C85814CAA82758257B0
:0D413700C00212407FD0028A8212407FA891
:0A4144004C181818868212407FE51F
:0A414E004C24FCF8868212407F1218
:0541580040BAD04C222A
:0E415D00AA82AB83758200C002C0031240F339
:0C416B00E5827877F274D0C0E07582E540
:0C417700124107AC8215817878ECF274DC
:0E41830082C0E07582E5124107AC821581789A
:0B41910079ECF27483C0E07582E51247
:0C419C004107AC821581787AECF2748443
:0D41A800C0E07582E5124107AC82158178F8
:0B41B5007BECF27485C0E07582E5121F
:0C41C0004107AC821581D003D002787C4E
:0E41CC00ECF28A048B02C004C00275829012CD
:0741DA00412D158115812222
:0C41E1007879E2C0E07482C0E07582755D
:0C41ED0012412D15811581787AE2C0E0A6
:0E41F9007483C0E075827512412D1581158109
:0C420700787BE2C0E07484C0E075827532
:0C42130012412D15811581787CE2C0E07D
:0E421F007485C0E075827512412D15811581E0
:0C422D007878E2C0E074D0C0E0758275C3
:0C42390012412D158115817877E2C0E05C
:09424500758274124107158122F3
:0E424E00AA82C0027582741241071581758222
:0A425C00F01240F37582A30240F354
:0C4266007582E01240F37582A30240F361
:0E42720053F4C743F62043901843FE1853FE42
:02428000DF223B
:024282007A14AC
:0442840000DAFD223D
:0C428800AA82C002124282D002C01D8A2D
:074294008212406015812237
:0C429B00AA82C002124272751D387582A2
:0C42A70038124288D00274204AFB8B1DA4
:0E42B300758238C002C00312428890000A12C1
:0E42C1001F097430C0E075823812406015810C
:0B42CF00D0038B1D75823812428875E9
:0C42DA001D30758238124288D002742812
:0C42E6004AF51D75823812428890000ACB
:0342F200021F099F
:0642F50075820002429BED
:0642FB0075821002429BD7
:0A43010012039D7806E2B40A0122BF
:09430B001204537807E2700A78ED
:0943140000E2F58212407F80E412
:01431D00227D
:09431E001204537807E260012249
:0C4327007800E2FA08E2FBC3E49A74019B
:094333009B500678077402F22287
:04433C007C007D0084
:0E434000C3EC9AED9B5042EC4D601BEC540711
:0E434E00701675820AC002C003C004C00512BA
:0A435C0016AFD005D004D003D00244
:0E436600C002C003C004C0051240BA120369B1
:0E4374007582201216AFD005D004D003D002FF
:074382000CBC00BA0D80B76E
:0643890075820A0216AF66
:0C438F001204537800E2FA08E2FBC002BE
:0C439B00C003120453D003D0027800E2EB
:0A43A700FC08E2FD7807E260012245
:0E43B1008C828D83C002C00312415DD003D008
:0343BF00027C007D
:0943C2008A058B061ABAFF011BE3
:0E43CB00ED4E602E8C050CED540770127582BD
:0E43D9000AC002C003C0041216AFD004D00305
:0243E700D00202
:0E43E900C002C003C004124266120369D00471
:0643F700D003D00280C5D6
:0943FD001241E175820A0216AFBB
:0C4406001204537800E2FA08E2FBC00246
:0C441200C003120453D003D0027800E273
:0A441E00FC08E2FD7807E2600122CD
:0E4428008C828D83C002C00312415DD003D090
:014436000283
:094437008A048B051ABAFF011B6F
:0E444000EC4D6032C002C0031202FAE582C4E5
:0E444E0054F0FCC0041202FAAD82D004D00378
:0B445C00D002ED42047807E26001226C
:0E4467008C82C002C00312424ED003D00280ED
:01447500C185
:034476000241E11F
:06447900907B1B0207739B
:027B1B00F54231
:027B1D00377BB4
:027B1F001E4303
:027B2100467BA1
:027B23008F438E
:027B2500597B8A
:027B2700064412
:027B2900827B5D
:027B2B00014314
:027B2D00AC7B2F
:027B2F00FB4217
:067B3100C27B0000000011
:0E7B37004400456E61626C652064656275678E
:017B4500003F
:0E7B460047203C636F756E743E0047657420E7
:057B5400646174610092
:0E7B590049203C636F756E743E203C6164648D
:0E7B6700723E00496E707574203C636F756E3F
:0D7B7500743E206174203C616464723E0027
:0E7B82004F203C636F756E743E203C6164645E
:0E7B9000723E004F7574707574203C636F7503
:0E7B9E006E743E206174203C616464723E008F
:0E7BAC0050203C627974653E202E2E2E005033
:087BBA00757420646174610020
:087BC200520052657365740066
:0C447F00AA82AB837405B53F0E75820263
:0B448B00C002C0031215F4D003D002E1
:08449600AC3F053FEC2CFD24B6
:0A449E00FFF582E434F6F583EAF03E
:0E44A800A3EBF0EC701FF5D1C2C043B8017A4F
:0644B600D77BF68BD57ADE
:0644BC00D77BF68AD47ADA
:0644C200DF7BF68BD37ACC
:0544C800DF7BF68AD243
:0344CD008C8222BC
:0C44D000AA828AF005F07B017C008006C7
:0644DC00EB2BFBEC33FCAE
:0E44E200D5F0F7ADD67E00ED5203EE5204EB9E
:0D44F0004C600A758202C0021215F4D00261
:0C44FD00EAC40354F8FA24D7F582E43432
:06450900F6F583AB40ACA7
:0A450F00418C05EDF0EA24D7FAE430
:0C45190034F6FD8A828D83A3EBF08A82C9
:0A4525008D83A3A3AB42AC438C06C8
:0E452F00EEF08A828D83A3A3A3EBF08A828D27
:0C453D0083A3A3A3A3E545F08A828D832D
:0C454900A3A3A3A3A3E544F074062AF585
:0C45550082E43DF583E546F074072AF58A
:0B45610082E43DF58374084547F0221A
:0A456C00AA828AF005F074018002B3
:0245760025E03E
:0E457800D5F0FBFBF4FC52D1EB55D6600D7470
:0C458600804BF5D6000000000000000093
:0A459200EA2A24FFF582E434F6F56E
:0E459C0083E0FAA3E0FC8A828C83E4F08BD6E5
:0A45AA0000000000000000000022E5
:0A45B400AA828AF005F0740180026B
:0245BE0025E0F6
:0645C000D5F0FB42D722FA
:0A45C600AA828AF005F07401800259
:0245D00025E0E4
:0E45D200D5F0FBFA74804AF5D6EAF452D122F5
:0C45E000C022C0E0C0F0C082C083C00256
:0E45EC00C003C004C005C006C007C000C00167
:0B45FA00C0D075D0007A017B007C006F
:0C460500C3EC953F5033EA55D16026C24B
:0C461100C0EAF4F5D1EB2B24FFF582E4A5
:0C461D0034F6F583E0FDA3E0FE8D828EF4
:0D462900837401F08D828E83121E7780084D
:08463600EA2AFA0C8C0380C78C
:0E463E00D0D0D001D000D007D006D005D004D7
:0D464C00D003D002D083D082D0F0D0E0D0D7
:0246590022320B
:0C465B00AA82C2AFEA75F003A42409F59E
:0C46670082E434F7F5837401F090F70949
:06467300121E77D2AF22F7
:09467900AA82D20010AF02C200B7
:0E46820090F70FC002123E68D002EA75F003F6
:0A469000A4FB2409F582E434F7F5D9
:0A469A0083E0FCEB2409FBE434F795
:0E46A400FD8B828D83A3E0FE8B828D83A3A30A
:0C46B200E0FBA20092AFEB7006EC60078A
:0346BE00EE700497
:0446C10075820222DA
:0946C5007BAC7C0DBA00028005FB
:0546CE00BA0114800A8E
:0A46D30090F719E0FBA3E0FC80085B
:0846DD0090F71BE0FBA3E0FCD9
:0E46E500C3EB94E8EC64809483500475820368
:0146F30022A4
:0E46F400C374589B749B8CF063F08095F0505B
:05470200047582012294
:044707007582002295
:0C470B00E582FA75F003A4FB2409FCE42D
:0C47170034F7FD8C828D83A3A37401F0A5
:0C47230090F1CEE0FC600ABC0102802F87
:05472F00BC0270804D8A
:05473400BA000280053F
:05473900BA01668010CA
:0E473E00D2A3900005C003121F09D003C2A32E
:02474C00805497
:0E474E00D2A4900005C003121F09D003C2A41C
:02475C00804497
:0E475E00BA0041D2A3900005C003121F09C289
:0D476C00A39000C8121F09D2A490000512EE
:084779001F09D003C2A4802136
:0E478100BA011ED2A3900005C003121F09C288
:0D478F00A39000C8121F09D2A490000512CB
:06479C001F09D003C2A4B6
:0A47A200EB2409FBE434F7FA8B82E4
:0747AC008A83A3A3E4F022BD
:0347B300120AC225
:0847B60090F709121E397A0088
:0C47BE00EA24FE40F3EA75F003A4FB249B
:0A47CA0009FCE434F7FD8C828D83B6
:0A47D400E06052EB2409FBE434F727
:0647DE00FC0BBB00010C06
:0E47E4008B828C83E0703EEA701890F1C3E087
:0E47F200FB6011EB75F064A4F58285F083C0C6
:0648000002121F09D002A4
:0E4806008A82C00212470B9000C8121F09D010
:0B48140002EA75F003A42409FBE43461
:0A481F00F7FC8B828C83A37401F078
:034829000A809270
:07482C0012039D907BCA12EC
:074833000564E5827001221B
:0A483A0012039D7806E2B46D1090A1
:0D4844007BCF120564E582600675820102DB
:02485100470B13
:0A4853007806E2B46410907BD412E2
:0C485D000564E582600675820002470BCE
:0648690078077402F22240
:06486F00C04C85814C12D3
:0E4875004679E5822582FA907BDB93CAA393F5
:0C488300FB7C80E54C24FCF886050886D0
:0E488F00067F80C002C003C004C005C006C082
:0A489D000774E3C0E0747BC0E07410
:0D48A70080C0E0126CDAE58124F7F581D0C5
:0248B4004C2294
:0A48B60074D4C0E0747BC0E075828A
:0C48C0000012486F1581158174CFC0E014
:0C48CC00747BC0E075820112486F1581FA
:0348D80015812225
:0E48DB00C2A343FF0853F5F7C2A443FF1053D6
:0348E900F5EF22C6
:0848EC001248DB7408C0E074FF
:0848F4007CC0E074B3C0E07465
:0748FC0047C0E090F71D1218
:0C4903001C15E58124FCF581907BFC0272
:02490F0007732C
:057BCA00446F49740046
:057BCF006D61696E000C
:077BD40064726F6775650024
:027BDB00107C1C
:027BDD00187C12
:027BDF001E7C0A
:027BE100257C01
:0E7BE30049676E697465723A20253673205327
:0B7BF10074617475733A2025730A005C
:027BFC002C4813
:027BFE002A7CDF
:027C0000B64884
:067C0200657C000000009B
:087C080069676E697465720082
:087C1000756E6B6E6F776E005C
:067C180072656164790051
:077C1E0061637469766500E3
:057C25006F70656E00A8
:0E7C2A0069203C6B65793E207B6D61696E7C44
:0E7C380064726F6775657D004669726520692C
:0E7C4600676E697465722E203C6B65793E2076
:0E7C5400697320646F69742077697468204436
:037C6200264900B0
:0E7C65007400546573742069676E69746572EB
:017C73000010
:09491100AA82787DE25A4290224C
:0C491A00AA82787DE25202EAF452902258
:0C492600AA82787DE2F4FBE59052037851
:074932007DE25A4BF59022D3
:09493900AA82787DE25A62902204
:0A494200C04C85814CAA82C002120D
:0C494C004911E54C24FCF88682088683A3
:0B495800121F09D0028A8212491AD0F7
:024963004C22E4
:0C496500AA82787DEAF2EAF4FB52F4EB3F
:064971005290EA42FE2212
:0C4977007582011249117880E2603690D0
:07498300F7E3E07030756EF0
:03498A002E756F18
:05498D00F87880E2F55E
:0549920070757100903A
:06499700F7E61251E29068
:07499D00F7E37880E2F090DF
:0B49A400F7E4E0FA0A90F7E4EAF0788C
:0749AF0080E4F290F82E12E3
:0249B6001E776A
:0E49B800744CC0E090F7E2124CBF158175827E
:0449C6000102491A87
:0E49CA00E4C0E0744EC0E090F794124D36AA9F
:0B49D8008215811581EA7003F5822230
:0C49E30090F7E1E0FA20E7047582002262
:0849EF00740724B3F56EE434F3
:0449F700F1F56F75F2
:0649FB007008E4F5719064
:0A4A0100F7D812523BE582601C7AE0
:044A0B00747B7C8AB2
:044A0F006E8B6F75C6
:064A13007007E4F571904C
:0D4A1900F1BA12523BE58260047582002262
:0E4A260090F795E0FABAFF1890F796E0FB784B
:084A340081F290F797E0FC907D
:0A4A3C00F7E4F090F7E5EBF0805A84
:0C4A4600EA605790F796E0FB7881E224CC
:084A520001FCEBB50402800732
:074A5A0090F926E0FB603F2C
:0A4A6100787F797EE2F5F0E3B5F00E
:094A6B003474042494F56EE43463
:044A7400F7F56F8A59
:054A7800707571009053
:064A7D00F86E1251E27810
:084A83007FE4F290F795E07862
:084A8B007EF290F796E0FA7844
:084A930081F290F7E5EAF090D2
:054A9B00F2C5121E77B8
:0B4AA00090F926E4F090F797E0FA9000
:0E4AAB00F7E4E0FBEAB5030B90F7E3E4F090CC
:054AB900F7E2121E7778
:044ABE0075820122DA
:024AC200AA82C6
:0C4AC4007880E2B4401390F925E0FB601C
:0D4AD0000C90F82EC002121E39D00280E7B3
:0C4ADD0090F925E0FB60147880E2FB7883
:0A4AE9008004F2EB242EF582E43481
:054AF300F8F583EAF074
:014AF800229B
:0B4AF90090F925E0FA700490FFFF2206
:0A4B0400787F797EE2F5F0E3B5F06A
:054B0E000490FFFF22EE
:0A4B1300787FE2FA787F04F2EA24CA
:0A4B1D006EF582E434F8F583E0FA47
:074B27007B008A828B8322D0
:077C74004E3043414C4C006F
:0E4B2E009000A4E493FA740193FB90F7E2EA7E
:0D4B3C00F090F7E374FFF090F9267401F09B
:0E4B490090F925E0FA60281249CAE58260F270
:084B570074442494F56EE4346B
:044B5F00F7F56F7582
:064B63007008E4F57190FA
:064B6900F8261251E2786B
:094B6F00167401F212497780D19D
:034B7800021F1504
:0E4B7B0090F925E0FA702290F9257401F0748B
:084B89007BC0E0747CC0E07405
:084B91002EC0E0744BC0E0905F
:0B4B9900F8AE121C15E58124FCF5812C
:014BA40022EE
:0C4BA50090F925E0FA601B90F925E4F07F
:0E4BB10090F8AEE0FAA3E0FB4A600B124DF55F
:084BBF00900001121F0980EAB9
:014BC70022CB
:0C4BC800AA82C002E4C0E0C0E074C2C0D9
:094BD400E0744AC0E0904AF912B5
:0E4BDD0017B5E58124FCF581D002EA600302E1
:024BEB004B7B02
:014BED0022A5
:067C7B00736C61766500E8
:0C4BEE00C022C0E0C0F0C082C083C00242
:0E4BFA00C003C004C005C006C007C000C00153
:0E4C0800C0D075D000539BFCE5E930E50812E2
:074C16004DF553E9DF8014A6
:0E4C1D00E5E930E40F90F9297401F090F929CF
:064C2B00121E7753E9EFB1
:0E4C3100D0D0D001D000D007D006D005D004DE
:0D4C3F00D003D002D083D082D0F0D0E0D0DE
:024C4C00223212
:024C4E007A00EA
:034C5000BA0E0099
:0D4C53005018EA907CDF93FB7CDFEA0490B0
:0D4C60007CDF93FD8B828C83F00A0A80E3D9
:014C6D002224
:094C6E0090DF3BE0FABA010122DB
:0E4C770075E104121D0790DF3BE0FABA01F26E
:014C8500220C
:0B4C8600AA82C002120AC290F92B1291
:0D4C91001534124C6ED00290DF06E4F09056
:0D4C9E00F1D0E0FBA3E0FCA3E0FDA3E0905B
:0E4CAB00DF09EDF090DF0AECF090DF0BEBF08C
:064CB90090DF02EAF02288
:0A4CBF00C04C85814CAA82AB83A88B
:0B4CC9004C1818188682C002C00312AD
:0C4CD4004C86D003D00290F929E4F09047
:0A4CE000F927E0FCA84C181818860C
:054CEA00447545008A3D
:044CEF00408B417540
:064CF30042D97543DF7594
:084CF90046137547428C82123C
:094D010044D090F927E0F582127C
:0B4D0A00456C75E103D21010AF02C22F
:014D1500108D
:0B4D160090F929E0FA700C90F929C018
:054D210022121E39D032
:034D26002280EDFB
:084D2900A21092AF90F92B12C9
:054D31001592D04C2298
:0A4D3600C04C85814CAA82AB83902B
:0C4D4000F92AE4F0A84C181818E624FE2C
:0E4D4C00F582C002C003124C86D003D0029044
:0A4D5A00F927E0FCA84C1818188691
:054D64004475450075D7
:064D690040D97541DF8A0C
:044D6F00428B4375BB
:084D730046137547128C8212F1
:094D7B0044D090F927E0F5821202
:0C4D8400456C75E102E54C24FCF8E6608B
:0C4D900010E54C24FCF886027B008A82AF
:054D9C008B83121EB024
:074DA100D21010AF02C21096
:0E4DA80090F928E0FA701590F92AE0FA700EE2
:064DB60090F928C0221252
:084DBC001E39E582D02260E4FB
:0A4DC400A21092AFE54C24FCF8E6C3
:054DCE006003121EFC51
:0E4DD30090F928E0FA700C90F927E0F58212B2
:054DE10045C6124C6EF6
:074DE60090F92B12159290C9
:084DED00F928E0F582D04C2208
:0A4DF50090F92A7401F090F92802E9
:024DFF001E771D
:0C4E010090F92AE4F075827D124C869036
:064E0D00F929E4F07A002F
:034E1300BA0E00D4
:0D4E16005018EA907CD193FB7CDFEA0490F9
:0D4E23007CD193FD8B828C83F00A0A80E322
:014E3000225F
:0D4E310090F927E0F58212456C75E103D27F
:064E3E000110AF02C201E9
:0E4E440090F929E0FA700F90F92AE0FA700850
:084E520090F929121E3980EAD3
:0C4E5A00A20192AF90F929E0FA700C90D0
:094E6600F927E0F5821245C6129D
:024E6F004C6E87
:074E7100124C4E90F92B02D8
:024E7800159291
:094E7A00124E0190F927E0FA7BC9
:044E8300ED7C7C8BBB
:044E8700408C4175A5
:064E8B0042D97543DF75FA
:064E9100447DE4F54575C7
:084E970046137547028A8212DE
:054E9F0044D0024E3179
:0E4EA400AA82C002124E01D00290F927E0FB54
:0C4EB2007403C39AC42354E024EFFAE414
:064EBE00347CFC8A408CEC
:054EC400417542D975A3
:074EC90043DF754478E4F5B6
:054ED000457546137555
:084ED50047428B821244D00217
:024EDD004E3154
:0A4EDF0090F92A7401F090F92902FD
:024EE9001E7732
:0E4EEB00E582FA602190F92CE0FAA3E0FB4A80
:0E4EF9007031124BA57582FF124C8675E103D5
:0A4F070090F92C7401F0E4A3F022ED
:0E4F110090F92CE0FAA3E0FB4A6010124C6EFF
:074F1F0090F92B121592908E
:064F2600F92CE4F0A3F0F9
:014F2C002262
:0C4F2D007A02C00212039DD0027806E256
:054F3900B40A0280072C
:074F3E001204AC7802E2FA54
:0E4F45000AEA30E10A758201C002124EEBD07A
:014F5300025B
:0A4F5400BA0325C00274A7C0E07480
:0C4F5E007DC0E07480C0E0126CDA1581A8
:0E4F6A001581158112171A12174875820A1246
:044F780016AFD0029E
:0A4F7C00EA30E006758200024EEBF9
:014F86002208
:024F87007A00AE
:034F8900BA50001B
:0D4F8C005018EA907C8193FB7CDFEA0490D2
:0D4F99007C8193FD8B828C83F00A0A80E3FB
:0A4FA600124C4E90F9287401F0122D
:0E4FB000447FE58290F927F075E90075913095
:094FBE00439A01907DC2020773C1
:0E7C810027C028C029C02AC02BC02CC02DC08F
:0E7C8F002EC0070608000DA30E110FA2101143
:0E7C9D0006001B101A561CE91D0A1E001F1FB0
:0E7CAB0023812435250900D3019103240444CC
:0E7CB90005001207133014181500166017038B
:0A7CC700180019002F0030003100F2
:0E7CD1000CD60D5E0E900F021116030004007B
:0E7CDF000CDA0DA30E110FA21136032404447B
:027CED00550040
:0E7CEF00000000000000000000000000000087
:0E7CFD00000000000000000000005555555525
:0E7D0B00555555550000000000000000000016
:0E7D190000000000000000000000000000005C
:0E7D27005555555555555555000000000000A6
:0E7D3500000000000000000000000000000040
:0E7D430000000000555555555555555500008A
:0E7D5100000000000000000000000000000024
:0E7D5F00000000000000000000000000000016
:0E7D6D00000000000000000000000000000008
:0E7D7B000000000000000000000000000000FA
:0E7D89000000000000000000000000000000EC
:0E7D97000000000000000000000000000000DE
:027DA5000000DC
:0E7DA7004869742061206368617261637465CD
:0D7DB5007220746F2073746F702E2E2E00DC
:027DC2002D4F43
:067DC400CA7D0000000072
:0E7DCA0043203C312073746172742C203020F1
:0E7DD80073746F702C206E6F6E6520626F7476
:0E7DE600683E00526164696F206361727269C9
:087DF4006572207465737400D0
:0200A00002005C
:0200A200FDFF60
:0200A40000005A
:0400A600331B1200F6
:0C4FC700C022C0E0C0F0C082C083C00265
:0E4FD300C003C004C005C006C007C000C00176
:0E4FE100C0D075D00090F930E0FA7B000ABA1B
:034FEF0000010BB3
:0E4FF20053021F7B0090F931E0FC7D00EAB510
:085000000406EBB50502801C5B
:0A50080090F930E02432F582E43420
:0C501200F9F583E5F9F090F930E0045462
:06501E001FFA90F930F0CA
:0E50240090F930121E77D0D0D001D000D00706
:0E503200D006D005D004D003D002D083D082A7
:07504000D0F0D0E0D02232D5
:0E50470090F952E0FA90F953E0FBEAB503014C
:015055002238
:0E50560090F974E0FA702290F9747401F090F1
:09506400F953E02454F582E43410
:0C506D00F9F583E0F5F990F953E00454E4
:065079001FFA90F953F04C
:01507F00220E
:0C508000C022C0E0C0F0C082C083C002AB
:0E508C00C003C004C005C006C007C000C001BC
:0D509A00C0D075D000C2EA90F974E4F012A5
:0650A700504790F952127F
:0E50AD001E77D0D0D001D000D007D006D0059D
:0E50BB00D004D003D002D083D082D0F0D0E059
:0350C900D02232C0
:0550CC00D310AF01C389
:0250D100C0D04D
:0E50D30090F930E0FA90F931E0FBEAB50308FD
:0850E10090F930121E3980EA3B
:0A50E90090F931E02432F582E4343E
:0C50F300F9F583E0FA90F931E004541F55
:0B50FF0090F931F08A82D0D092AF22ED
:05510A00D310AF01C34A
:04510F00C0D0AA82E0
:0C51130090F952E0FB7C000BBB00010C8B
:0E511F0053031F7C0090F953E0FD7E00EBB5BA
:0E512D000510ECB5060C90F952C002121E39A6
:04513B00D00280D44A
:0A513F0090F952E02454F582E434A4
:0C514900F9F583EAF090F952E004541FDD
:0C51550090F952F0125047D0D092AF22D7
:05516100D310AF01C3F3
:02516600C0D0B7
:0E51680090F952E0FA90F953E0FBEAB5030229
:025176008008AF
:0851780090F952121E3980E883
:05518000D0D092AF2227
:0E518500AA82C002125161D002EA24FB50013E
:0151930022F9
:0E51940043FB80EA2AFA907DFC93F5FAEA24A8
:0A51A200FCFAE4347DFB8A828B8363
:0651AC00A3E493F5FC22D0
:0E51B200AAF174FD5AF5F0740245F0F5F1AA69
:0E51C000F5749F5AF5F0744045F0F5F543F490
:0E51CE00C075F8C075820012518575FB8243D2
:0651DC00A808439A082216
:0A7DFC00A307A308A3093B0B3B0CEF
:0851E200AA82AB83AC70AD7131
:0951EA008C068D071CBCFF011DA1
:0A51F300EE4F601FAE6EAF6F8E82AC
:0E51FD008F83E0F88A828B83F00ABA00010BE0
:0A520B0074012EF56EE43FF56F808C
:01521500D4C4
:015216002275
:08521700AA82AB83AC6FAD70FD
:09521F008C068D071CBCFF011D6B
:0C522800EE4F600E8A828B83E56EF00A68
:06523400BA00E80B80E562
:01523A002251
:08523B00AA82AB83AC70AD71D7
:095243008C068D071CBCFF011D47
:0C524C00EE4F60298A828B83E0FEAF6E7B
:0C525800A86F8F828883E0F9EEC399FEF6
:0552640060038E8222B0
:055269000ABA00010B70
:0A526E0074012FF56EE438F56F802F
:01527800CA6B
:045279007582002218
:0A527D00C04C85814CAA82AB8375FA
:03528700427875F5
:03528A0043F97570
:06528D0040C17541DFE5A0
:085293004C24FCF88644088657
:05529B004575460E758B
:0A52A0004701851F82C002C00312FF
:0A52AA0044D0D003D002851E828A92
:0452B400408B417575
:0652B80042C17543DFE571
:0852BE004C24FCF8864408862C
:0552C6004575460F755F
:0652CB0047411244D085AA
:0652D1001F8212456C85EE
:0652D7001E8212456C85E9
:0652DD001E821245B4D24E
:0652E3001010AF02C21022
:0A52E90090F976E0700C90F976C0A1
:0552F30022121E39D05B
:0352F8002280EE23
:0752FB00A21092AFD04C227B
:07530200C04C85814C85823F
:0553090042858343858D
:06530E001F827540C1750D
:0853140041DFE54C24FCF886A2
:05531C00440886457500
:06532100460E7547111253
:0953270044D090F97874FFF07590
:035330004078754D
:0353330041F975C8
:0653360042C17543DFE5F2
:08533C004C24FCF886440886AD
:055344004575460F75E0
:065349004701851E8212DF
:06534F0044D0851F82120C
:06535500456C851E82126A
:06535B00456C851E821264
:0853610045B4D21010AF02C2E6
:015369001033
:0A536A0090F976E0700C90F976C01F
:0553740022121E39D0D9
:035379002280EEA1
:07537C00A21092AFD04C22F9
:0E538300AAF174FE5AF5F0740145F0F5F143FD
:0E539100F43875864075C20075C53190F97705
:08539F0012447FE582F51E9027
:0853A700F97612447FE582F55E
:0253AF001F22BB
:0301BC00754A0180
:0553B100D310AF01C3A1
:0A53B600C0D0854882854983D0D01D
:0353C00092AF2287
:0C53C300C022C0E0C0F0C082C083C00265
:0E53CF00C003C004C005C006C007C000C00176
:0A53DD00C0D075D00074012548F51A
:0553E70048E43549F522
:0453EC0049054BE53F
:0553F0004AB54B0675F3
:0553F5004B00123E64B4
:0E53FA00D0D0D001D000D007D006D005D0040E
:0D540800D003D002D083D082D0F0D0E0D00D
:02541500223241
:05541700D310AF01C33A
:0A541C00C0D085824A754B00D0D045
:0354260092AF2220
:0E54290075E40075DB7575DA3075E50475E61F
:0E5437000075E70075E200D2DED2B975E4061A
:015445002244
:0354460053C6BF8B
:0B544900E5BE30E6FB43BE0453C6C0C6
:08545400E5C6543F600280F838
:01545C00222D
:0D545D0090DE077421F090DE097410F090CD
:06546A00DE0B7404F022C9
:0C547000C022C0E0C0F0C082C083C002B7
:0E547C00C003C004C005C006C007C000C001C8
:0D548A00C0D075D000C2E890DE02E0FA78D4
:0A54970084E24AF27884E2540160D6
:0754A1000690F979121E7755
:0B54A8007884E25420600690F9F012B6
:0254B3001E7762
:0E54B50090DE04E0FA30E40690F2C5121E7795
:0B54C30090DE06E0FA30E20312545DB8
:0E54CE00D0D0D001D000D007D006D005D00439
:0D54DC00D003D002D083D082D0F0D0E0D039
:0254E90022326D
:0E54EB0090DE0EE4F090DE11E0FA30E10122D6
:0A54F900788AE2FB24DF50027B20DA
:075503007A02BB20028006C2
:06550A007A0A7886E4F243
:06551000788AE2C39BF261
:0C5516008B041BEC60287887E2FC08E2A4
:0E552200FD08E2FE8C828D838EF01272A0FFD7
:0C553000788774012CF2E43D08F208EECC
:08553C00F290DE20EFF080D2B6
:0B55440090DE0EE4F090DE11EAF02291
:08554F00AA82AC837BAA7D0057
:0E5557008B828D83E493FE60408B828D83A354
:0E556500E493FFB504278A071AEF7021BC02F9
:0C5573000E8B828D83A3A3E493FF788A43
:03557F00F28004B3
:04558200788AEEF243
:0C5586007887EBF208EDF2087480F22246
:0E5592008B828D83E493FE2BFBE43DFD80B7FE
:0155A00022E8
:0C55A10090DE0EE4F090DE16E0FA788D4B
:0955AD00C3E29A5004788DE2FA81
:0655B600788DE2C39AF2B9
:0C55BC008A031AEB601D788EE2FB08E207
:0C55C800FC90DE20E0FD8B828C83F078EC
:0B55D4008E74012BF2E43C08F280DD35
:0155DF0022A9
:0A55E000AA82788AE2FB788A04F2BE
:0755EA00EB248BF8EAF2222A
:0C55F100AA8278857401F290DE00EAF0D6
:0155FD00228B
:0D55FE0090DE0E7405F090DE107408F09041
:0D560B00DE12E04401F090DE0E7404F09019
:0C561800DE137408F090DE157401F0221F
:07562400788E74F4F20874A3
:08562B00F9F2788D7408F21207
:0856330055A1788DE26001220F
:0A563B007887748BF208E4F208741B
:0C56450060F2788AE4F290F9F4E0FA7464
:0B565100605AFB6009BB2003025719E0
:03565C00025749A9
:08565F0053021FBA0002800F84
:06566700BA01030256E047
:06566D00BA02030257021D
:0356730002574992
:0C56760090F9F5E0FA6017BA05028021F7
:05568200BA0602802BB6
:05568700BA08028038A2
:05568C00BA0902803E96
:0356910002574974
:0D5694007582001255E07582001255E0028B
:0256A100574967
:0D56A30090F9F6E0FAA3E08A821255F102B8
:0256B000574958
:0D56B20090F9F6E0FAA3E0FB8A828B8312E8
:0556BF00554F025749A0
:0956C4007890E2F5821255E00233
:0256CD0057493B
:0C56CF0090F9F6E0FAA3E07890EAF212FD
:0556DB0055FE025749D5
:0C56E00090F9F5E0FA6005BA0A5F800E50
:0E56EC007582001255E07582001255E0804F65
:0856FA007582001255E08047A3
:0957020090F9F5E0FA6002803E26
:0E570B007582001255E07582001255E0803064
:0A57190090F9F5E0FABA20028005CD
:05572300BA21238010F3
:08572800788D7407F2788E748D
:0857300060F20874FDF2801123
:08573800788A7407F278877487
:0957400060F20874FDF208E4F2C5
:0B57490090DE0EE4F0788AE260277822
:0B575400867401F290DE117440F090AA
:0C575F00F9FAE0FAA3E0FB788AE2FC7D96
:0C576B0000C3EA9CEB9D5004788AEAF22F
:035777000254EBEE
:0A577A00788DE2600C78867402F26C
:0757840090DE117440F022D9
:0C578B0090F9FAE0FAA3E0FB4A600C7809
:0B579700867403F290DE117460F022B3
:0B57A2007886E4F290DE117448F022DB
:0457AD007886E4F224
:0757B100D20210AF02C20298
:0A57B8007884E2540160087884E26E
:0557C20054FEF2800816
:0857C70090F979121E3980E906
:0C57CF00A20292AF90DE0EE4F090DE111A
:0C57DB00E0FA30E40A90DE117480F078EF
:0357E70086E4F263
:0C57EA00EA30E20990DE11E4F07886E479
:0157F600F2C0
:0C57F7007886E2B4010BEA20E107C00252
:055803001254EBD0027D
:0C580800EA30E0A57886E2B400028008D7
:085814007886E2B402978005DA
:05581C001256248090EB
:0C5821001255A190DE0EE4F0788DE270CC
:0C582D000D7886E4F290DE117448F00261
:0258390057B165
:09583B0090DE117440F00257B137
:0E58440090DE0E7405F090DE11E0FA30E00800
:0858520090F9F0121E3980EA02
:01585A00222B
:0E585B0090DE0E7405F090DE11E04401F09036
:0C586900F9F0E0FAA3E0FB7882EAF20814
:0A587500EBF290F9F0E4F0A3F0224A
:05587F00D310AF01C3CE
:09588400C0D07885E2700280209A
:0C588D0090F9F0E0FAA3E0FB4A700F78FD
:0C58990082E2B4400708E2B40002800282
:0258A50080067B
:0658A70012584412585B88
:0558AD00D0D092AF22F3
:0558B200D310AF01C39B
:0B58B700C0D0AA827885E27002802930
:0D58C200C002125844D00290DE2AEAF09095
:0E58CF00F9F0E02401F0A3E03400F090F9F0CD
:0E58DD00E0FAA3E0FBBA4006BB000312585BE2
:0558EB00D0D092AF22B5
:0E58F00090F9F2E0FAA3E0FB4A704290DE0E5F
:0E58FE007404F090DE14E0FA20E00490FFFF46
:01590C002278
:0E590D0090DE17E0FB7A0090DE16E0FC7D00D5
:0E591B004202ED420390F9F2EAF0A3EBF0EA4B
:0E5929004B701190DE0E7404F090DE14E0540A
:06593700FEF090FFFF22CC
:0D593D0090F9F2E024FFFAA3E034FFFB90A4
:0D594A00F9F2EAF0A3EBF090DE28E0FA900D
:0E595700F9F2E0FBA3E0FC4B700E90DE0E7444
:0A59650004F090DE14E0FB54FEF0A5
:07596F007B008A828B83227A
:02597600C2AFBE
:0E5978001258F0AA82AB838A048B05BAFF0B8B
:0B598600BBFF0890F2C5121E3980E73D
:05599100D2AF8C822260
:0D59960043BE801255FE12545D439A0290EC
:0D59A300DE06E4F090DE04F090DE02F0225B
:0E59B00090DE07E4F090DE09F090DE0BF0537D
:0E59BE009AFD90DE06E4F090DE04F090DE022A
:0559CC00F053BE7F2234
:0859D1001259967406C0E0743F
:0859D9007EC0E074ADC0E07473
:0759E10057C0E090F97912B4
:0C59E8001C15E58124FCF581747FC0E0F3
:0959F4007458C0E074B2C0E07404
:0759FD0058C0E09058F012C1
:095A040017B5E58124FCF58122AF
:047E0600757362002E
:077FEA0000C20100000008C5
:0B5A0D00AA8290F9FCEAF090F9FD7805
:0B5A180011E2F01253B1AA82AB8390A0
:0E5A2300F9FEEAF0A3EBF09000A4E493FA740D
:0E5A31000193FB90FA00EAF0A3EBF090F36C07
:0E5A3F00E0FAA3E0FB90FA02EAF0A3EBF0908D
:0B5A4D00FA047848E2F0A308E2F090B1
:0B5A5800FA067846E2F0A308E2F090A6
:0B5A6300FA087844E2F0A308E2F078B3
:0C5A6E0014E2FA08E2FB90FA0AEAF0A346
:0D5A7A00EBF07410C0E0E4C0E090F9FC1205
:075A8700527D1581158122FB
:0E5A8E0090F97512153475C52DC292758201FE
:0E5A9C00125A0D7406C0E0E4C0E090FA0C123D
:0C5AAA00530215811581D29290F97512FB
:0B5AB600159290FA0CE0FAA3E0FB90C0
:0E5AC100FA0EE0FCA3E0FDECF4FCEDF4FDEACF
:0B5ACF00B50408EBB50504740180016C
:015ADA00E4E7
:035ADB00F582222F
:0E5ADE0090F97512153475C52DC292758202AD
:075AEC00125A0D90FA2A1274
:0E5AF300153490FA11E075F002A4FAABF0C081
:0E5B010002C00390FA12125302158115819012
:085B0F00FA2A121592D29290BD
:055B1700F97502159272
:0E5B1C0090F97512153475C52DC2927582036D
:095B2A00125A0DD29290F9750295
:025B33001592C9
:0E5B350090F36CE0FAA3E0FB4A700890F36C6A
:055B4300121E3980ED87
:025B48007A00E1
:035B4A00BA0A0094
:0E5B4D005019900064C002121F09125A8EAB4C
:0C5B5B0082D0027891EBF2EB70030A801C
:015B6700E25B
:0C5B68007891E2602790FA10E0FA7B00D0
:0C5B74008A828B83121EB07A117BFF8A9C
:0E5B8000828B83121E39E5826005125ADE8088
:015B8E00D93D
:055B8F00125B1C80D434
:035B9400021F15D8
:0B5B97007891E2FA7B00C002C00374AA
:0A5BA2000AC0E0747EC0E07480C009
:0C5BAC00E0126CDAE58124FBF5817891B1
:045BB800E270012274
:0E5BBC0090FA11E0FA7B0090FA10E0FC7D00F8
:0E5BCA0090FA0CE0FEA3E0FFC002C003C0048E
:0B5BD800C005C006C0077421C0E074C7
:0C5BE3007EC0E07480C0E0126CDAE58146
:065BEF0024F7F5817A00A5
:0D5BF50090FA11E0FBC3EA9B5030EA2A242D
:0A5C020012F582E434FAF583E0FBAA
:0C5C0C00A3E0FCC002C003C0047451C03F
:0C5C1800E0747EC0E07480C0E0126CDA22
:0B5C2400E58124FBF581D0020A80C658
:0A5C2F007456C0E0747EC0E074807B
:0C5C3900C0E0126CDA1581158115812283
:0E5C4500D29243FE0453F4FB907E5812077374
:095C53007460C0E0747EC0E074CE
:085C5C0035C0E0745BC0E0906C
:0C5C6400FA2B121C15E58124FCF58122AE
:0E7E0A00436F6D70616E696F6E2072756E6EE3
:097E1800696E673A2025640A0036
:0E7E21006465766963653A2025640A757064AD
:0E7E2F0061746520706572696F643A20256485
:0E7E3D000A6368616E6E656C733A2025640AF4
:067E4B00646174613A005D
:057E510020253575003D
:027E56000A0020
:027E5800975B36
:067E5A006A7E000000003A
:0A7E6000636F6D70616E696F6E0054
:0E7E6A004C00436F6D70616E696F6E206C6925
:0A7E78006E6B207374617475730063
:085C7000E54F60047A0A80058B
:055C78001250CCAA82CD
:065C7D00EA624E8A4D228E
:065C8300AA4DBA2C01221B
:045C8900BA2A012210
:045C8D00BA0A01222C
:055C9100125C7080EDC3
:075C9600AA4DBA2C028008A0
:055C9D00BA2E02800395
:035CA200BA2A0318
:035CA500025C702E
:015CA80022D9
:0E5CA900AA827B00C002C003125C96D003D01A
:0C5CB70002742DB54D0D7B01C002C0032E
:075CC300125C70D003D00257
:075CCA007C007D0075500015
:0A5CD100C3E5509A503FAE4DBE30BF
:015CDB0000C8
:0A5CDC004038EE24C640338C6E8D74
:0B5CE6006F90000AC002C003C006124D
:0E5CF1006B3DAF82A883D006EE24D079002F41
:0B5CFF00FCE938FD0550C004C0051290
:0C5D0A005C70D005D004D003D00280BB38
:0A5D1600EB6007C3E49CFCE49DFD74
:055D20008C828D83223E
:085D2500125C967A0075500033
:0A5D2D0074FE25504040AB4D8B047E
:035D3700BB30007E
:0B5D3A004009EB24C640047BD0801A17
:035D4500BC41005E
:0B5D48004009EC24B940047BC9800C2A
:035D5300BC610030
:095D5600401BEC249940167BA9C6
:0C5D5F00EAC454F0FDEB2C4DFA0550C0D6
:085D6B0002125C70D00280BA44
:035D73008A8222FF
:0A5D7600C04CE581F54C2408F581CE
:0C5D8000125CA9E5828583F078D7F20858
:0E5D8C00E5F0F2758202125CA9AA82AB837860
:0A5D9A00D9EAF2AA4DBA2E3775823D
:0C5DA40004125CA9E5828583F078DAF235
:045DB00008E5F0F220
:0A5DB40074FC2550402D78DAE2F56A
:095DBE006E08E2F56F90000A1274
:0C5DC7006B3DE5828583F078DAF208E598
:065DD300F0F2055080DB38
:0B5DD90078DAE4F208F2BA2C02800332
:035DE400754F01F7
:085DE70078D7E2F56E08E2F541
:055DEF006F75700075E6
:0C5DF400710090968075F098E4126BA787
:0C5E0000A84C08A68208A68308A6F0089B
:075E0C00F678D9E2F56E758E
:065E13006F0075700075C0
:0C5E19007100902710E4F5F0126BA7A8B0
:0C5E25004C0808080808A68208A683089C
:0C5E3100A6F008F678DAE2FC08E2FDE4D6
:0A5E3D00FAFBE54C2405F8EC26F50D
:0A5E47006EED0836F56FEA0836F537
:0A5E510070EB0836F571900032E4A2
:0D5E5B00F5F0126BA7AA82AB83ACF0FD75C9
:065E68006E03E4F56FF586
:0A5E6E0070F5718A828B838CF0EDD1
:0C5E7800126C15AA82AB83ACF0FDA84CA4
:0E5E840008EA26FAEB0836FBEC0836FCED08BF
:0B5E9200368A828B838CF0854C81D017
:025E9D004C2295
:0E5E9F00AA827B00C002C003125C96D003D022
:0A5EAD0002E551B54D047B01800BA6
:085EB700EAB54D047B008003F5
:035EBF00754F011B
:0A5EC200C003125C70D0038B822233
:075ECC00AA4DBA2A02801260
:055ED300BA0A02800D77
:055ED800BA0D02800874
:085EDD00125C70125C8380E787
:0B5EE500BA2A17742A654EFAC0021298
:0B5EF0005D25AB82D002EAB503012261
:045EFB00754F0122BC
:045EFF00754F0122B8
:0C5F03001253B1E5828583F07894F20817
:0A5F0F00E5F0F278B6E24420FA78DB
:0C5F19009BEAF2758202125CA9AA827851
:0C5F2500A9EAF2758202125CA9AA827837
:0C5F3100AAEAF2758202125CA9AA82782A
:0A5F3D00ABEAF2125C8375820212D7
:0C5F47005D76AA82AB83ACF0FD789EEA88
:0C5F5300F208EBF208ECF208EDF27551D8
:0C5F5F005375824E125E9FE58260277829
:0C5F6B009EE2FA08E2FB08E2FC08E2FDFE
:0E5F7700C3E49AFAE49BFBE49CFCE49DFD78F5
:0C5F85009EEAF208EBF208ECF208EDF2E4
:0E5F9100758203125D76AA82AB83ACF0FD78B8
:0C5F9F00A2EAF208EBF208ECF208EDF2C6
:0C5FAB00755157758245125E9FE58260BB
:0C5FB7002778A2E2FA08E2FB08E2FC08EE
:0E5FC300E2FDC3E49AFAE49BFBE49CFCE49D3F
:0C5FD100FD78A2EAF208EBF208ECF208FE
:025FDD00EDF2E3
:0E5FDF007582FF125CA9AA82AB83BA010B780F
:0A5FED009BE2FB430310789BEBF2EC
:0E5FF7007582FF125CA9AB82AC838B02EA2498
:05600500F050027A0FCB
:0A600A00789BE2FBEA4203789BEB6F
:0E601400F2125C707582FF125CA9AB82AC8345
:0E6022008B02EA24E6401EEA75F00AA4FA7426
:0C6030002EB54D15758201C002125CA94E
:0B603C00AB82AC83D002EB2AFA80029A
:026047007AFFDE
:0860490078ADEAF2125C8378E5
:0C605100AFE4F27582FF125CA9AA82ABDA
:0C605D0083789CEAF208EBF2125C8312DC
:076069005ECCE54F703E9094
:06607000FAA312153490A2
:0C607600FAA2E04401F07894E2FA08E29B
:0A608200FB7892EAF208EBF27A963E
:0A608C007B004303F08A6E8B6F75F2
:066096007020E4F571909A
:06609C00FAA41251E2908B
:0660A200FAA31215929012
:0560A800FAA2021E77C0
:0160AD0022D0
:0E60AE00758201125CA9AA82758201C00212DD
:0C60BC005CA9AB82AC83D002BB0104786D
:0360C800BCE4F243
:0860CB00EAB503047401800131
:0160D300E4E8
:0B60D400FCC004125C70125C83D0045E
:0760DF00742AB54D02807028
:0760E600740AB54D02806948
:0760ED00740DB54D02806245
:0C60F40078BCE2FB758202C003C00412FD
:0E6100005CA9AD82AE83D004D0038D02BB0C2F
:01610E000090
:0C610F00E433FD6008EB2BFE24BDF8EA31
:01611B00F291
:0D611C00C003C004C005125C70125C831249
:096129005C70125C8375820212A5
:0E6132005CA9AE82AF83D005D004D0038E02EC
:0C614000ED609CEB2B24BDFD04F8EAF29E
:0A614C00EA60900B78BCEBF280894A
:0C615600C004125ECCD004E54F60057858
:04616200BCE4F22285
:0A616600EC603090FAA3121534909B
:0C617000FAA2E04402F07AB77B0043037F
:06617C00F08A6E8B6F75C6
:066182007020E4F57190AD
:06618800FAC41251E2907E
:06618E00FAA31215929025
:05619400FAA2021E77D3
:0161990022E3
:05619A00125C837A088D
:0E619F00C002125C70125C83D002DAF47582CA
:0E61AD0002125CA9AA82758202C002125CA9CD
:0E61BB00AB82758202C003125CA9AC82C004E4
:0C61C900125ECCD004D003D002E54F7071
:0A61D5001178A6ECF278A7EBF2783F
:0861DF00A8EAF278B67440F260
:0161E7002295
:0661E800AA82AB83AC5259
:0E61EE008C051CED60388A828B83E493FDA340
:0E61FC00AA82AB83BDA016900032C002C00381
:0E620A00C004C005121F09D005D004D003D077
:016218000283
:0E6219008D82C002C003C00412510AD004D00E
:0562270003D00280C25B
:01622C00224F
:07622D00754E00754F0012D1
:096234005C707447B54D02800155
:01623D00223E
:0A623E00125C707450B54D0280012F
:016248002233
:08624900125C70AA4DC00212A4
:076251005C70AB4DC00312AD
:076258005C70AC4DC00412A4
:0C625F005C70D004D003D002742CB54D4C
:06626B0029E4BA4701041A
:0C627100FD6009BB4706BC4103025F034F
:0C627D00ED6009BB5306BC56030260AE86
:0C628900BA5209BB4D06BC430302619AE7
:0162950022E6
:0D6296007582011251859000C8121F097514
:0662A300521A907E8212E7
:0262A90061E8AA
:0B62AB001250CCAA82BA240312622D0C
:0862B600E55360F11250CC1217
:0862BE0058B290F930E0FA90AB
:0D62C600F931E0FBEAB503E812171A80E396
:0E62D300AA82900032C002121F09D0028A82F5
:0962E100125185900032021F09E0
:0A62EA007553017511017582001251
:0662F400541775520B90D7
:0962FA007E9C1261E8758200121D
:0663030062D375520B90FD
:096309007E9C1261E87582041209
:0263120062D354
:0863140012597612510A80F8BB
:09631C0074B3C0E0747EC0E074AB
:0863250096C0E07462C0E09034
:0C632D00FAE4121C15E58124FCF58190B7
:056339007EA7020773BE
:0E7E8200A0A100090801000100010000000994
:0C7E90000D0AA0A100033C00003C0D0AFC
:0B7E9C00A0A1000405000500000D0A75
:027EA7003E6338
:027EA900B77EA2
:027EAB00EA6289
:067EAD00C57E000000008C
:047EB3006770730081
:0E7EB7006700446973706C6179204750530076
:0E7EC500550055706461746520475053206667
:087ED30069726D7761726500B0
:07633E0090FAA31215349040
:0E634500FAB6E0FA7B0090FAB5E0FC7D00901D
:0E635300FAB4E0FE7F00C002C003C004C00523
:0A636100C006C00774DBC0E0747EC4
:0E636B00C0E07480C0E0126CDAE58124F7F522
:0E6379008190FAB9E0FA7B0090FAB8E0FC7D62
:0E6387000090FAB7E0FE7F00C002C003C00421
:0B639500C005C006C00774F1C0E07432
:0C63A0007EC0E07480C0E0126CDAE58181
:0E63AC0024F7F58190FAB0E0FAA3E0FBA3E03D
:0E63BA00FCA3E0FD90FAACE0FEA3E0FFA3E040
:0E63C800F8A3E0F9C002C003C004C005C0067F
:0B63D600C007C000C0017407C0E074E5
:0C63E1007FC0E07480C0E0126CDAE5813F
:0E63ED0024F5F58190FAAAE0FAA3E0FBC002C5
:0A63FB00C0037419C0E0747FC0E015
:0E6405007480C0E0126CDAE58124FBF5819012
:0C641300FAA9E0FA7B00C002C00374226A
:0B641F00C0E0747FC0E07480C0E01299
:0E642A006CDAE58124FBF58190FAC9E0FA7B7B
:0A64380000C002C003742FC0E0741E
:0C6442007FC0E07480C0E0126CDAE581DD
:06644E0024FBF5817A0039
:0D64540090FAC9E0FBC3EA9B503EEA2A24FF
:0A646100CAFBE434FAFC8B828C8342
:0E646B00A3E0FD7E008B828C83E0FB7C00C0F2
:0C64790002C005C006C003C0047438C097
:0C648500E0747FC0E07480C0E0126CDAAC
:0B649100E58124F9F581D0020A80B8F3
:0A649C00743FC0E0747FC0E074801C
:0E64A600C0E0126CDA15811581158190FAA301
:0364B4000215923C
:0E7EDB00446174653A20253032642F25303220
:087EE900642F253032640A0009
:0E7EF10054696D653A20253032643A253032EE
:087EFF00643A253032640A00E8
:0E7F07004C61742F4C6F6E3A20256C6420255F
:047F15006C640A008E
:097F1900416C743A2025640A0051
:0D7F2200466C6167733A20307825780A00BC
:097F2F00536174733A20256400CB
:077F380020256420256400F0
:077F3F000A646F6E650A0081
:0901BF0078EA74FFF20874FFF203
:0C64B70090F97512153475C531C2919032
:0C64C300FB5C743DF090FB5D742AF090CF
:0E64CF00FB5E7480F090FB5F74A6F07404C056
:0E64DD00E0E4C0E090FB5C12527D1581158159
:0864EB00D29190F9750215929F
:0C64F30090F97512153475C531C29190F6
:0D64FF00FB5C74D7F07401C0E0E4C0E090D5
:0E650C00FB5C12527D158115817401C0E0E424
:0E651A00C0E090FB5C12530215811581D291F6
:0765280090F9751215929025
:06652F00FB5CE0F5822296
:0665350078EEE260012295
:07653B0090FB5B12153478A0
:08654200EEE2600690FB5B0233
:02654A001592A8
:0E654C001264F3E582FA20E00DC0021264B77B
:08655A007582091215F4D0024C
:0965620053023CBA0C030265E689
:05656B00BA1402806279
:05657000BA1C02804985
:05657500BA2402803091
:05657A00BA2C0280179D
:0A657F00BA347878EF7409F278DC82
:0D658900E4F208F2087440F208E4F2806ABF
:0A65960078EF7409F278DCE4F208F3
:0A65A000F2087420F208E4F28056BD
:0A65AA0078EF7408F278DCE4F208E0
:0A65B400F2087410F208E4F28042CD
:0A65BE0078EF7408F278DCE4F208CC
:0A65C800F2087408F208E4F2802ED5
:0A65D20078EF7408F278DCE4F208B8
:0A65DC00F2087404F208E4F2801AD9
:0A65E60078EF7408F278DCE4F208A4
:0A65F000F2087402F208E4F28006DB
:0665FA007582091215F480
:0C66000078EFE2F5F005F07A017B0080F5
:01660C000687
:06660D00EA2AFAEB33FB60
:0B661300D5F0F778F0EAF208EBF2781F
:0B661E00F2EA24FFF2EB34FF08F278F0
:0B662900F0E2FC08E2FD7E007F00783C
:0C663400E0ECF208EDF208EEF208EFF2E4
:0C66400078DCE2C39CFC08E29DFD08E24F
:0C664C009EFE08E29FFF78E4ECF208EDEF
:0C665800F208EEF208EFF278E8EAF2082F
:0B666400EBF278EE7401F290FB5B0299
:02666F00159282
:0566710078EDE2600C71
:0C6676001264F3E58230E7F878EDE4F2FE
:0166820022F5
:0766830012667190F9751217
:0E668A00153475C531C29190FB5C7482F078B6
:0C669800EFE2FA7B007410C39AFAE49B56
:0C66A4008AF005F078EAE2FA08E2FB80D8
:0166B00007E2
:0766B100C3EB13FBEA13FA2F
:0C66B800D5F0F690FB5DEAF078EAE2FA1B
:0C66C40078EFE224F8F5F005F0EA80021F
:0266D00025E0C3
:0E66D200D5F0FB90FB5EF090FB5FE4F07404EB
:0E66E000C0E0E4C0E090FB5C12527D15811515
:0C66EE008178E0E2FA08E2FBC002C00381
:0D66FA0090FB6012527D15811581D29190A8
:06670700F97512159278ED
:05670D00ED7401F22211
:0767120012667190F9751287
:0E671900153475C531C29190FB5C7403F078A5
:0C672700EFE2FA7B007410C39AFAE49BC6
:0C6733008AF005F078EAE2FA08E2FB8048
:01673F000752
:07674000C3EB13FBEA13FA9F
:0C674700D5F0F690FB5DEAF078EAE2FA8B
:0C67530078EFE224F8F5F005F0EA80028F
:02675F0025E033
:0E676100D5F0FB90FB5EF090FB5FE4F074045B
:0E676F00C0E0E4C0E090FB5C12527D15811585
:0B677D008178F0E2C0E008E2C0E0908C
:0C678800FB6012530215811581D2919024
:05679400F975021592E9
:0967990078ECE2600712668378D7
:0367A200ECE4F232
:0167A50022D1
:0C67A600AA82AB8378EAE2B5020608E2A2
:0467B200B503012208
:0C67B600C002C003126799D003D0027823
:0967C200EAEAF208EBF2026712A8
:0A67CB00C04C85814CC082C083C021
:0B67D500F0C0E078EFE2F5F005F0A85E
:0C67E0004C08860608860708860208861A
:0367EC0003800D1A
:0D67EF00C3EB13FBEA13FAEF13FFEE13FEEA
:0E67FC00D5F0F090FB5BC006C007121534D03C
:0A680A0007D006E54C24FAF879F0F7
:0E68140086F0E3B5F00A0886F009E3B5F0025D
:026822008009EB
:096824008E828F831267A6801298
:0C682D00C006C007126799D007D006789B
:06683900EAEEF208EFF2A6
:0C683F0078F2E2FA08E2FB7C007D00A881
:0C684B004C08E6520208E6520308E65230
:0C6857000408E65205EA2460F582EB34E8
:09686300FBF583E54C24FCF886EA
:05686C006E08866FE5D7
:086871004C24FAF88670088639
:05687900711251E278EC
:08687E00EC7401F290FB5B12C7
:096886001592758201854C81D048
:02688F004C2299
:0A689100C04C85814CC082C083C05A
:0B689B00F0C0E078EFE2F5F005F0A897
:0C68A6004C088606088607088602088653
:0368B20003800D53
:0D68B500C3EB13FBEA13FAEF13FFEE13FE23
:0E68C200D5F0F090FB5BC006C007121534D075
:0C68D00007D0068E828F831267A678F234
:0C68DC00E2FA08E2FB7C007D00A84C08FA
:0E68E800E6520208E6520308E6520408E652A1
:0868F60005EA2460F56EEB34A5
:0468FE00FBF56FE552
:086902004C24FAF886700886A7
:0A690A0071E54C24FCF88682088633
:08691400831251E290FB5B12BB
:09691C001592758201854C81D0B1
:026925004C2202
:0769270090FB5B1215341216
:06692E00679990FB5B027B
:026934001592BA
:0E693600AA82AB83ACF0FD90FB5BC002C003F5
:0E694400C004C005121534126799D005D004A6
:0C695200D003D00278EFE2F5F005F080F1
:01695E000D2B
:0D695F00C3ED13FDEC13FCEB13FBEA13FA80
:0B696C00D5F0F078EAEAF208EBF275D3
:066977006EFF78F0E2F56E
:06697D006F08E2F57090C6
:06698300FB6012521778C0
:08698900EC7401F290FB5B12BB
:066991001592758201223F
:0769970012653590FB5B1255
:0E699E0015341264F3AA827B00C002C0037499
:0A69AC0046C0E0747FC0E07480C0B4
:0C69B600E0126CDAE58124FBF58178EF3B
:0C69C200E2FA7B00C002C003745CC0E07D
:0C69CE00747FC0E07480C0E0126CDAE559
:0C69DA008124FBF58178F0E2C0E008E2C7
:0A69E600C0E07473C0E0747FC0E0ED
:0E69F0007480C0E0126CDAE58124FBF581783A
:0A69FE00F2E2C0E008E2C0E0748994
:0B6A0800C0E0747FC0E07480C0E012AA
:0C6A13006CDAE58124FBF58178DCE2C040
:0E6A1F00E008E2C0E008E2C0E008E2C0E07477
:0A6A2D009FC0E0747FC0E07480C0D9
:0E6A3700E0126CDAE58124F9F58190FB5B0238
:026A45001592A8
:096A4700D29143FE0253F4FD223A
:0E7F4600466C617368207374617475733A2021
:087F54003078253032780A0074
:0E7F5C00466C61736820626C6F636B20736803
:097F6A006966743A2025640A00DE
:0E7F7300466C61736820626C6F636B207369EB
:087F81007A653A2025640A002C
:0E7F8900466C61736820626C6F636B206D61E3
:087F9700736B3A2025640A0017
:0E7F9F00466C617368206465766963652073C3
:0A7FAD00697A653A20256C640A0029
:0400000002015F3268
:03000B00023E842E
:0100130032BA
:03001B00024FC7CA
:0100230032AA
:01002B0032A2
:0300330002547004
:01003B003292
:030043000245E093
:03004B000253C39A
:01005300327A
:01005B003272
:01006300326A
:01006B003262
:03007300025080B8
:01007B003252
:03008300024BEE3F
:0301C800020086AC
:05008600126A5080FE2B
:0A6A50001248DB1254467582011251
:0C6A5A00496575820112491120930878EB
:046A6600167401F2AF
:036A6A003093FD69
:076A6D00125429123FFD1233
:066A7400404A12088112E5
:066A7A005383121C0C12F4
:066A800023D71230F312CF
:066A860037B71259D112CE
:066A8C0051B212631C125E
:066A92001517123D0D1264
:096A98004F87758200124BC812F1
:066AA10048EC12447912DA
:066AA7005C4512125E02C4
:026AAD001FAD1B
:087FB700312E3600000000002D
:0E7FBF00616C7475736D657472756D2E6F72E2
:027FCD0067004B
:0E7FCF0054656C654D657472756D2D76312E9E
:027FDD00300072
:0E00AA001201100102000020FEFF0B000001F9
:0E00B8000102030109024300020100C03209E7
:0E00C6000400000102020100052400100105E3
:0E00D400240101010424020205240600010794
:0E00E2000581030800FF09040100020A000066
:0E00F0000007050402400000070585024000DD
:0E00FE000004030904200361006C0074007507
:0E010C000073006D0065007400720075006DD8
:0E011A00002E006F0072006700200354006585
:0E012800006C0065004D0065007400720075EB
:0E013600006D002D00760031002E0030000E0E
:0E014400033000300030003000300031000089
:056AAF007A10E4FBFC7D
:0E6AB400E58225E0F582E58333F583EB33FBC5
:0A6AC200EC33FCEB956EF5F0EC955B
:096ACC006F4006FCABF0438201AF
:036AD500DADD22E5
:086AD800FB7A20E4FCFDFEFF47
:0E6AE000E5822582F582E58333F583E5F03308
:0B6AEE00F5F0EB33FB4017DAE98042C3
:0E6AF900E5822582F582E58333F583E5F033EF
:056B0700F5F0EB33FB8B
:0E6B0C00EC33FCED33FDEE33FEEF33FFEC9582
:066B1A006EED956FEE9593
:086B200070EF95714013EC9534
:086B28006EFCED956FFDEE958A
:096B300070FEEF9571FF43820134
:026B3900DABEC2
:026B3B00EB224B
:06018E00E478FEF6D8FD46
:08016C007907E94400601B7AE9
:0501740001907FEA7814
:030179006075931B
:0A017C00FDE493F2A308B8000205A9
:0801860093D9F4DAF27593FF3E
:0B6B3D00E582856EF0A4C582C0F085E3
:0A6B48006FF0A4D0F025F0C583859E
:086B52006EF0A42583F58322F7
:086B5A00E56E456F60467A010B
:076B6200E56E25E0F56EE58C
:096B69006F334012F56FE58295CF
:0A6B72006EE583956F40030A80E68C
:036B7C00C3E56FFF
:076B7F0013F56FE56E13F53D
:016B86006EA0
:0A6B8700C3E582956EF5F0E58395F5
:086B91006F4005F58385F082D9
:076B9900C3E56F13F56FE582
:066BA0006E13F56EDAE150
:016BA60022CC
:0C6BA700AAF0FBE582856EF0A4FCADF0C6
:0C6BB300E583856EF0A42DFDE435F0FEB6
:0C6BBF00E582856FF0A42DFDE5F03EFEA0
:0C6BCB00E433FFEA856EF0A42EFEE5F036
:0C6BD7003FFFE583856FF0A42EFEE5F083
:0C6BE3003FFFE5828570F0A42EFEE5F077
:0B6BEF003FFFEB856EF0A42FFFEA854E
:0A6BFA006FF0A42FFFE5838570F013
:0C6C0400A42FFFE5828571F0A42F8EF014
:056C10008D838C82223F
:0801940078F4E84400600A79E8
:03019C0000759358
:06019F00F0E4F309D8FCB6
:0801A500786CE8440C600C7951
:0B01AD000D90F0F4E4F0A3D8FCD9FAA8
:0E6C1500FBC2D530E715D2D5E4C39582F582D7
:0D6C2300E49583F583E495F0F5F0E49BFB28
:0A6C3000E57130E717B2D5E4C39513
:056C3A006EF56EE4950B
:056C3F006FF56FE49504
:056C440070F570E495FD
:036C490071F57171
:0E6C4C00EB126AD830D513FBE4C39582F582B3
:0C6C5A00E49583F583E495F0F5F0E49BED
:016C6600220B
:0A6C6700AA82AB83ACF07D007E0032
:0E6C71008A828B838CF01272A0FF60258F82C6
:056C7F000ABA00010B40
:0E6C8400C002C003C004C005C0061216AFD087
:0E6C920006D005D004D003D0020DBD00D20EF6
:026CA00080CFA3
:0E6CA20075820AC005C0061216AFD006D005D6
:066CB0008D828E83A322F9
:02008B00E4731C
:066CB600C04C85814C1268
:056CBC0016AFD04C22D0
:086CC10085826485836585F07E
:056CC90066E4F561F531
:046CCE0062F5638583
:036CD20054679074
:056CD5006CB6026D9A8F
:066CDA00C04C85814CE571
:076CE0004C24FBF567E4F50D
:046CE70061F562F5FC
:076CEB0063E54C24FBF88671
:066CF200640886650886B7
:056CF80066906CB6126D
:056CFD006D9AD04C224D
:076D0200AA82C057C058C06F
:066D0900597419C0E0748A
:066D0F006DC0E0C055C09C
:046D1500568A8222F6
:0A6D1900158115811581055FE4B5B1
:046D23005F020560A6
:016D27002249
:0E6D2800AA8274302AFA24C6500A74072AFA86
:066D3600300303430220BC
:056D3C008A82026D02D5
:0E6D4100E582FAC4540FF582C002126D28D00C
:096D4F0002740F5AF582026D284E
:066D580085826EAB5AAC0F
:046D5E005BAD5CAE1F
:046D62005DAF5E754E
:026D66006F209C
:0E6D6800EF2FFFEE235401FA4207EB2BFBEC5A
:0C6D760033FCED33FDEE33FEC3EF956EF1
:0A6D82004008EFC3956EFF430301C4
:066D8C00D56FD98B5A8C73
:046D92005B8D5C8E2B
:046D96005D8F5E228D
:076D9A0085825585835685B3
:036DA100615785B2
:036DA400625885AD
:046DA7006359E4F553
:036DAB005FF56031
:056DAE00AA64AB65AC16
:0C6DB300668A828B838CF01272A0FD7443
:096DBF00012AF564E43BF5658C42
:086DC80066EDFA70030272810E
:056DD000BA250280035A
:036DD500027279CE
:056DD800C204C205C267
:046DDD0006C207C221
:046DE10008C209C219
:046DE5000AC20B755E
:086DE90068007569007DFFAE32
:046DF10064AF65AB7B
:016DF5006637
:0E6DF6008E828F838BF01272A0FAA3AE82AF52
:066E0400838E648F658B94
:0B6E0A0066BA25078A82126D0280998B
:056E15008A04BC3000FE
:0D6E1A00402A8A04EC24C64023BDFF13E586
:0B6E27006975F00AA4FCEA24D02CF5E9
:076E32006970C1D20580BDAB
:0D6E3900ED75F00AA4FCEA24D02CFD80B019
:0A6E4600BA2E07BDFFAA7D0080A64A
:056E50008A04BC610092
:0D6E5500400E8A04EC248540075302DFD272
:036E6200038002A8
:026E6500C20366
:056E6700BA2002805575
:056E6C00BA2B02804B6F
:056E7100BA2D02804172
:056E7600BA4202804B4E
:056E7B00BA4302805043
:066E8000BA440302702B6E
:066E8600BA460302704150
:066E8C00BA490302702B5D
:056E9200BA4C0280343F
:066E9700BA4F0302703245
:066E9D00BA5003026FC2AF
:056EA300BA5302804C0F
:066EA800BA550302703729
:066EAE00BA580302703C1B
:036EB40002704524
:056EB700D204026DF69B
:056EBC00D206026DF694
:056EC100D207026DF68E
:056EC600D209026DF687
:056ECB00D20A026DF681
:086ED00030090AE56714F88897
:056ED800678602800F37
:0A6EDD00E56724FEF88867860308C5
:056EE7008604188B0277
:086EEC008A82126D0202704E51
:0A6EF400E56724FDF88867860308AF
:0A6EFE00860408860618188B5A8CCB
:046F08005B8E5C85BB
:066F0C005A82855B8385BB
:0C6F12005CF0C005127288AB82AC83D02A
:066F1E0005BDFF028B051A
:0A6F240020042CC3EB95695026E50C
:066F2E0069C39BF569AC8C
:016F340069F3
:0C6F35008C061C8C69EE6014758220C074
:0E6F410003C004C005126D02D005D004D003B9
:026F4F0080E4DC
:026F51008C6949
:026F53008D04AB
:076F5500855A82855B8385EC
:0C6F5C005CF01272A0FDFA602F8C051C86
:0E6F6800C374808DF063F08095F050208A8213
:0C6F7600C003C004126D02D004D003ADB3
:046F82005AAE5BAFF9
:066F86005C0DBD00010ED0
:056F8C008D5A8E5B8FA1
:036F91005C80C160
:066F940020040302704E10
:096F9A00C3EB9569400302704E3F
:076FA300E569C39BF569AC31
:016FAA00697D
:0B6FAB008C051C8C69ED700302704C1B
:0C6FB600758220C004126D02D00480E936
:0A6FC200E56724FDF88867860508DE
:0A6FCC00860608860718188D5A8EF5
:046FD6005B8F5CADC4
:046FDA005CBD80001A
:066FDE0040047A43801418
:036FE400BD60008D
:066FE70040047A50800B0B
:036FED00BD4000A4
:066FF00040047A49800212
:026FF6007A58C7
:0E6FF8008A82C002126D0275823A126D027515
:0E7006008230126D02758278126D02D002BACD
:047014004902800BA2
:05701800BA50028006E1
:06701D00855B82126D414B
:08702300855A82126D418023A1
:07702B00D20875680A801C01
:057032007568088017DD
:0570370075680A8012DB
:05703C00756810800DD5
:04704100D20B8009E5
:077045008A82126D02800235
:02704C008C694D
:09704E00300B5AE56724FCF888B8
:0C70570067860408860508860608860780
:087063001818188C5A8D5B8E81
:04706B005C8F5D7564
:03706F005ADF7570
:037072005B7F75CC
:027075005C803D
:04707700855A6B8546
:03707B005B6C85C6
:05707E005C6D740125AA
:077083006BFFE4356CFCAD6E
:04708A006D8F5A8C20
:04708E005B8D5C8535
:067092006B82856C838512
:0A7098006DF01272A0FCFA70030202
:0270A2006DAED1
:0770A4008A82126D0280CC0C
:0770AB00E5687003026DAE01
:0470B200756A773054
:0770B600092BE56714F888BF
:0A70BD0067E6FD3395E0FEFFFC8D51
:0470C7005A8E5B8FF3
:0470CB005C8C5D205C
:0A70CF00085EAC5A7D007E007F00D1
:0570D9008C5A8D5B8E56
:0570DE005C8F5D804C99
:0970E300300A1FE56724FCF8885F
:0C70EC00678604088605088606088607EB
:0870F8001818188C5A8D5B8EEC
:057100005C8F5D802A98
:0A710500E56724FEF8886786040899
:0C710F00860518ED3395E0FEFF8C5A8DCC
:04711B005B8E5C8F9C
:05711F005D20080CAC2E
:087124005AAD5B7E007F008E76
:03712C005C8F5D18
:0A712F00300822E55D30E71BC3E4E1
:09713900955AFCE4955BFDE49518
:077142005CFEE4955DFF8C8B
:047149005A8D5B8E72
:05714D005C8F5D800273
:02715200C20871
:06715400D20CA86A7C00C9
:0A715A00755E00856882C004C00065
:0B716400126D58D000D004200C0DE587
:0A716F005EC4FDE6FE4DF618886AC6
:02717900800292
:02717B00A65E0E
:08717D000C8C03B20CE55A452D
:047185005B455C45C5
:087189005D70CE886A8C03E5FD
:067191006970037569013D
:0A719700200524200421EB04FCADC8
:0171A1006984
:0E71A200C3EC9D5015758220C003C004C005CB
:0C71B000126D02D005D004D0031D80E653
:0271BC008D69DB
:0C71BE0030080E75822DC003126D02D047
:0571CA0003156980239C
:0C71CF00EB602030060E75822BC003120E
:0871DB006D02D0031569800F5D
:0C71E30030070C758220C003126D02D032
:0371EF000315691C
:0571F200200424AC693B
:0B71F7008C051C8C69C3EB9D502B30F5
:0672020005047D3080024E
:027208007D20E7
:0E720A008D82C003C004126D02D004D0038038
:01721800DE97
:0A721900C3EB95695008E569C39BBB
:04722300F569800782
:05722700756900800202
:02722C008C696B
:02722E00A86A4C
:0A7230008B041BEC6026B20C200C4E
:0B723A000A08E6C4540FFC8C5E8007BD
:077245008604740F5CF55E86
:0C724C00855E82C003C000126D28D000D7
:04725800D00380D40B
:06725C00200403026DAEE8
:02726200AB6916
:097264008B041BEC7003026DAEFB
:0C726D00758220C003126D02D00380EB7C
:087279008A82126D02026DAE63
:07728100855F828560832216
:0B7FDF003C4E4F20464C4F41543E00EA
:04728800AA82AB83A8
:08728C001272A06003A380F858
:0C729400C3E5829AF582E5839BF5832216
:03015F0075817730
:0A01620012732AE582600302008692
:0E72A00020F71430F6148883A88220F507E644
:0672AE00A8837583002295
:0372B400E280F77E
:0372B700E493223B
:0272BA00E022D0
:0E72BC00C2D5E58330E70DD2D5E4C39582F547
:0672CA0082E49583F583C8
:0A72D000E56F30E70BE4C3956EF59F
:0572DA006EE4956FF564
:0172DF006F3F
:0E72E000126B5A30D50BE4C39582F582E4950B
:0372EE0083F583A2
:0172F100227A
:0E72F200C2D5E58330E70DD2D5E4C39582F511
:0673000082E49583F58391
:0A730600E56F30E70DB2D5E4C39542
:057310006EF56EE4952E
:037315006FF56FA2
:0E731800126AAF30D50BE4C39582F582E4957E
:0373260083F58369
:017329002241
:04732A007582002246
:00000001FF
